S01C00006376615F626F6F746C6F616465725F6D303132382E73726563AD
S1130000F0330020CDB800002B2E00003340000058
S113001000000000000000000000000000000000DC
S11300200000000000000000000000008F410000FC
S113003000000000000000008F420000F15C00009E
S113004014BD000014BD000014BD000014BD000068
S113005014BD000014BD000014BD000014BD000058
S113006014BD000014BD000014BD0000D95D0000E3
S1130070E15D000014BD000014BD000014BD0000CB
S113008014BD000014BD000014BD000014BD000028
S113009014BD000014BD000014BD000014BD000018
S11300A014BD000014BD0000A76D000014BD0000C5
S11300B014BD000014BD000014BD000014BD0000F8
S11300C044563032424C30313031000031353A350B
S11300D0363A313400000000446563203236203261
S11300E0303234000000000052502D3737410000F8
S11300F000000000000000000000000000000000FC
S113010000B5020093680120DB680340DBB2002BDA
S11301100AD093681B6A9B081840C0B2002803D019
S1130120D0690860012000E0002000BDF2B584B071
S11301300200002001009468E66801239E43012325
S11301400D00EDB21D403543E560049E3678002E67
S113015051D0D169294CA14201D2010012E0D169E8
S1130160274CA14201D219000CE0D169254CA142CF
S113017001D2022106E0D169234CA14201D203211C
S113018000E004210C00E4B2042C01D1002033E08F
S11301906C46617094680194019CE4680C25AC433E
S11301A06D466D78AD000C262E4026430396039CC5
S11301B0019DEC606C4620709068C4681025AC43C7
S11301C06D462D782D011026354025430295029C5D
S11301D0C4601C009568EE680127BE432700FFB287
S11301E01F403743EF609068006A8408180020407D
S11301F0C0B20028F7D0012005B0F0BD00093D00D1
S113020000127A0000366E01015A620200B5020043
S11302109068006A43081800C007C00FC0B20028E5
S113022003D090690860012000E0002000BDF2B511
S113023084B005000026A868012441692000084014
S1130240C0B2002868D0A868016A20000840C0B283
S1130250002861D0A8688069010920000840C0B264
S1130260002802D0012806D00BE001A92800FFF7DE
S1130270CDFF060005E001A92800FFF741FF0600B5
S1130280FFE73000C0B2002801D1002046E000940E
S1130290A8684069000A8007800FC0B2002805D012
S11302A0022808D004D3032808D00AE0009408E008
S11302B00220009005E00420009002E00820009055
S11302C0FFE7A868406940084006400EC0B2002815
S11302D002D18020039000E00390A8684069C00A1E
S11302E04007400FC0B2002802D10820029000E06D
S11302F00290A8684069800E27000740FFB27F1C67
S113030001980399484300997943029A514302F0B2
S113031034FD0499086026003000C0B205B0F0BD79
S1130320FCB502000020040095686E6901239E4319
S113033001232700FFB21F4037430197019E6E61DE
S11303401E006F463E704E78002E02D0012E0FD054
S11303501DE01C009568AF691026B743BC46260013
S1130360F6B2360110273E4067463E43AE6111E0C7
S113037004009568AF691026B743BC462600F6B260
S1130380360110273E4067463E43AE6102E004005A
S11303906D462C706C462478002C01D1002093E02B
S11303A0CC68012C01D104000FE0CC68022C01D1EF
S11303B01C000AE0CC68042C01D1022405E0CC68BE
S11303C0082C01D1032400E0FF242500EDB2FF2D09
S11303D001D1002078E06D466C7095686E69834F9A
S11303E03740BC466E4676783702C026B6003E409B
S11303F067463E436E614F88002F1CD04D88812D87
S113040019DA4D88802D01D1050000E04D889668E9
S11304100196019E7769FE26B743BC462E00F6B2CC
S11304207700FE263E4067463E43019F7E610F698A
S1130430002F02D11AE0002046E00D69092D15D2E3
S11304400D69082D00D0086995686E69B04F374072
S1130450BC460600F6B2F702E026B6013E40674607
S11304603E436E618F68012F02D104E000202BE02F
S11304708868022813D18868401E95686E69A54F64
S11304803740BC460600F6B2B6068027FF043E405D
S113049067463E436E610F78002F02D112E00020C0
S11304A012E0180095686E690127BE430700FFB289
S11304B01F4037436F619068056A18002840C0B236
S11304C00028F8D068460078F6BDF3B581B007007F
S11304D000242600009478690125C06901092800D8
S11304E00840C0B2002818D069463800FFF708FE5B
S11304F006003000C0B200280FD07869C069000A35
S11305004007400F85402900412905D2009802F098
S113051034FC0299086000E026003000C0B2FEBD41
S1130520FEB5020000206B4618706B465870536984
S1130530DE691024E443264010256F467F783F018E
S11305402F403743DF618E88012E01D103001EE066
S11305508B88022B01D1012319E08B88042B01D154
S1130560022314E08B88082B01D103230FE08B882E
S1130570102B01D104230AE08B88202B01D1052301
S113058005E08B88402B01D1062300E007231E00E1
S1130590F6B2072E17D06E46737056690196019E07
S11305A0F669A54F3740BC466E4676783702E0269A
S11305B0F6003E4067463E430296029E019FFE615E
S11305C001266F463E700E78002E01D0012600E011
S11305D006005769F86904403000C0B200010540C4
S11305E02543FD6168460078FEBD0000FFFCFFFF67
S11305F0F3B581B007000024260000947869012532
S11306008069010928000840C0B2002818D0694652
S11306103800FFF775FD06003000C0B200280FD087
S113062078698069000A4007400F85402900412904
S113063005D2009802F0A1FB0299086000E02600B0
S11306403000C0B2FEBDFEB5020000206B4618703B
S11306506B46587053699E691024E4432640102564
S11306606F467F783F012F4037439F618E88012E6C
S113067001D103001EE08B88022B01D1012319E074
S11306808B88042B01D1022314E08B88082B01D121
S113069003230FE08B88102B01D104230AE08B88FD
S11306A0202B01D1052305E08B88402B01D10623A3
S11306B000E007231E00F6B2072E17D06E467370B3
S11306C056690196019EB6695B4F3740BC466E463B
S11306D076783702E026F6003E4067463E430296AF
S11306E0029E019FBE6101266F463E700E78002E69
S11306F001D0012600E006005769B86904403000C3
S1130700C0B2000105402543BD6168460078FEBDC6
S1130710FFC7FFFFFFFFFFFBF3B581B00700002415
S113072026000094786901254069010928000840E1
S1130730C0B2002818D069463800FFF767FD0600EC
S11307403000C0B200280FD078694069000A400721
S1130750400F85402900412905D2009802F00DFB85
S11307600299086000E026003000C0B2FEBDFEB56C
S1130770020000206B4618706B46587053695E691E
S11307801024E443264010256F467F783F012F4014
S113079037435F618E88012E01D103001EE08B88F0
S11307A0022B01D1012319E08B88042B01D10223F0
S11307B014E08B88082B01D103230FE08B88102BC6
S11307C001D104230AE08B88202B01D1052305E005
S11307D08B88402B01D1062300E007231E00F6B2CC
S11307E0072E17D06E46737056690196019E76697E
S11307F0114F3740BC466E4676783702E026F60045
S11308003E4067463E430296029E019F7E6101265A
S11308106F463E700E78002E01D0012600E00600DF
S11308205769786904403000C0B20001054025438F
S11308307D6168460078FEBDFFF8FFFFF3B581B027
S11308400700002426000094786901250069010945
S113085028000840C0B2002818D069463800FFF7C5
S1130860D5FC06003000C0B200280FD078690069BA
S1130870000A4007400F85402900412905D200980D
S113088002F07BFA0299086000E026003000C0B252
S1130890FEBDFEB5020000206B4618706B46587012
S11308A053691E691024E443264010256F467F785F
S11308B03F012F4037431F618E88012E01D1030071
S11308C01EE08B88022B01D1012319E08B88042BB5
S11308D001D1022314E08B88082B01D103230FE0FC
S11308E08B88102B01D104230AE08B88202B01D1A3
S11308F0052305E08B88402B01D1062300E0072364
S11309001E00F6B2072E17D06E4673705669019614
S1130910019E3669A14F3740BC466E467678370251
S1130920E026F6003E4067463E430296029E019F43
S11309303E6101266F463E700E78002E01D00126DE
S113094000E006005769386904403000C0B2000175
S1130950054025433D6168460078FEBDF3B581B08E
S1130960070000242600009478690125406A0109E3
S113097028000840C0B2002818D069463800FFF7A4
S113098056FC06003000C0B200280FD07869406AD7
S1130990000A4007400F85402900412905D20098EC
S11309A002F0EBF90299086000E026003000C0B2C2
S11309B0FEBDFEB5020000206B4618706B465870F1
S11309C053695E6A1024E443264010256F467F78FD
S11309D03F012F4037435F628E88012E01D103000F
S11309E01EE08B88022B01D1012319E08B88042B94
S11309F001D1022314E08B88082B01D103230FE0DB
S1130A008B88102B01D104230AE08B88202B01D181
S1130A10052305E08B88402B01D1062300E0072342
S1130A201E00F6B2072E17D06E46737056690196F3
S1130A30019E766A594F3740BC466E467678370237
S1130A40E026F6003E4067463E430296029E019F22
S1130A507E6201266F463E700E78002E01D001267C
S1130A6000E006005769786A04403000C0B2000113
S1130A70054025437D6268460078FEBDF3B581B02C
S1130A80070000242600009478690125006A010902
S1130A9028000840C0B2002818D069463800FFF783
S1130AA0C6FB06003000C0B200280FD07869006A87
S1130AB0000A4007400F85402900412905D20098CB
S1130AC002F05BF90299086000E026003000C0B231
S1130AD0FEBDFEB5020000206B4618706B465870D0
S1130AE053691E6A1024E443264010256F467F781C
S1130AF03F012F4037431F628E88012E01D103002E
S1130B001EE08B88022B01D1012319E08B88042B72
S1130B1001D1022314E08B88082B01D103230FE0B9
S1130B208B88102B01D104230AE08B88202B01D160
S1130B30052305E08B88402B01D1062300E0072321
S1130B401E00F6B2072E17D06E46737056690196D2
S1130B50019E366A114F3740BC466E46767837029E
S1130B60E026F6003E4067463E430296029E019F01
S1130B703E6201266F463E700E78002E01D001269B
S1130B8000E006005769386A04403000C0B2000132
S1130B90054025433D6268460078FEBDFFF8FFFF2F
S1130BA070B504000E00002560690068000E80071F
S1130BB0800FC0B2002805D002280FD008D3032824
S1130BC012D017E031002000FFF720FB050011E0F0
S1130BD031002000FFF794FA05000BE031002000FB
S1130BE0FFF725FB050005E031002000FFF70EFBB1
S1130BF00500FFE72800C0B270BDF0B502004878D8
S1130C00012801D100230AE04878002801D10123FA
S1130C1005E04878022801D1022300E0FF231800F0
S1130C20C0B2FF2801D1002017E01C0050690668FB
S1130C30794D35402600F6B23704C026B6023E4050
S1130C402E43066050690068000E8007800F1C0068
S1130C50C0B2E4B2A042F5D10120F0BDF8B5040061
S1130C600E00002569462000FFF79AFF07003800B0
S1130C70C0B2002801D100200BE0E0680068010741
S1130C80090F0098C9B2491C02F077F830603800A7
S1130C90C0B2F2BD30B502008888002810D0888820
S1130CA011280DDA8C88641ED36818680F25A843B0
S1130CB02500EDB22D072D0F05431D60012000E036
S1130CC0002030BDF8B504000E0000256946200060
S1130CD0FFF7C4FF07003800C0B2002801D100208C
S1130CE00CE060690068000A0107090F0098C9B2A6
S1130CF0491C02F042F830603800C0B2F2BD70B551
S1130D0002008888002812D0888811280FDA8C887D
S1130D10641E53691D68414828402500EDB22E0227
S1130D20F0252D01354005431D60012000E0002021
S1130D3070BDF3B581B00500002426000094694617
S1130D402800FFF78BFF07003800C0B2002801D14C
S1130D5000201FE02869C821405801090800C00785
S1130D60C00FC0B2002812D02869C8214058000A18
S1130D700107090F0098C9B2491C01F0FEFF284978
S1130D80884201D0270003E00299086000E02700B0
S1130D903800C0B2FEBDF8B506000D000024009472
S1130DA069463000FFF75AFF002801D1002031E0E6
S1130DB0A88800282DD0A88811282ADA0098A988A4
S1130DC001F0DBFF1649884223D1A888401E31690F
S1130DD0C8228B58114A1A400300DBB21F02F023C9
S1130DE01B013B401343C8228B502A78002A01D0B0
S1130DF00124FFE73169C8200858102290432200DB
S1130E00D2B2120110231A400243C8200A50012012
S1130E1000E00020F2BD0000FFFFFCFFFFF0FFFF39
S1130E2000127A00F8B504000F00606940680109F7
S1130E300800C007C00FC0B2002801D100209BE009
S1130E40002005000090606907264068000C3040CF
S1130E50C0B2002843D160694068C00C3040C0B2C1
S1130E6000280BD0022815D00ED304281ED017D387
S1130E70062827D020D307282AD02FE0694620004F
S1130E80FFF757FF050066E069462000FFF738F9D1
S1130E90050060E069462000FFF7B8F905005AE054
S1130EA069462000FFF7C3F9050054E069462000B5
S1130EB0FFF7D4FE05004EE069462000FFF702FF6D
S1130EC0050048E069462000FFF7FFFA050042E00C
S1130ED069462000FFF720FC05003CE03BE0606928
S1130EE04068000C3040C0B201280AD033D3032834
S1130EF013D00CD305281CD015D3072825D01ED316
S1130F0029E069462000FFF729FD050023E0694632
S1130F10200000F03AFA05001DE06946200000F0C8
S1130F200DFA050017E06946200000F0E0F905001D
S1130F3011E06946200000F0EDFC05000BE0694675
S1130F402000FFF763F9050005E069462000FFF77C
S1130F505DF90500FFE72800C0B201280AD16069E5
S1130F604068000A064031000098C9B2491C01F0EB
S1130F7004FF38602800C0B2F2BDF2B582B00100AF
S1130F8001206A461070002002004B695C6810253D
S1130F90AC431500EDB22D011026354025435D60AC
S1130FA0029C6478002C40D0012C5DD0022C7AD0B5
S1130FB0032C00D1D4E0052C00D1F0E0072C00D1A3
S1130FC00CE10A2C00D18DE00B2C00D1A9E00C2CF3
S1130FD00CD00F2C00D12BE1102C00D11AE1112CD4
S1130FE000D109E1182C00D130E13DE102004B6948
S1130FF05D68B94C2C401500EDB22D04E026F602D4
S11310002E4026430196019C5C6004004D696E6885
S1131010B24F3740BC462600F6B2F704E026B603CA
S11310203E4067463E436E6021E102004B695D68C5
S1131030A94C2C401500EDB22D04E026F6022E40FA
S113104026430196019C5C6001244D696E68A34FA0
S11310503740BC462600F6B2F704E026B6033E400D
S113106067463E436E6002E102004B695D689A4C3C
S11310702C401500EDB22D04E026F6022E40264346
S11310800196019C5C6002244D696E68934F374061
S1131090BC462600F6B2F704E026B6033E40674697
S11310A03E436E60E3E002004B695D688A4C2C406D
S11310B01500EDB22D04E026F6022E4026430196DB
S11310C0019C5C6003244D696E68844F3740BC46C4
S11310D02600F6B2F704E026B6033E4067463E43D8
S11310E06E60C4E002004B695D687B4C2C401500C7
S11310F0EDB22D04E026F6022E4026430196019C13
S11311005C6004244D696E68744F3740BC46260009
S1131110F6B2F704E026B6033E4067463E436E60EF
S1131120A5E002004B695D686B4C2C401500EDB2E4
S11311302D04E026F6022E4026430196019C5C60B5
S113114005244D696E68654F3740BC462600F6B2EB
S1131150F704E026B6033E4067463E436E6086E0F1
S113116002004B695D685C4C2C401500EDB22D0407
S1131170E026F6022E4026430196019C5C6006247C
S11311804D696E68554F3740BC462600F6B2F704E9
S1131190E026B6033E4067463E436E6067E00200C9
S11311A04B695D684C4C2C401500EDB22D04E026D3
S11311B0F6022E4026430196019C5C6007244D698B
S11311C06E68464F3740BC462600F6B2F704E02668
S11311D0B6033E4067463E436E6048E001224B69D9
S11311E05D683D4C2C401500EDB22E04E025ED0267
S11311F0354025435D603AE002224B695D68364C18
S11312002C401500EDB22E04E025ED0235402543B7
S11312105D602CE003224B695D682F4C2C40150067
S1131220EDB22E04E025ED02354025435D601EE05D
S113123004224B695D68284C2C401500EDB22E0445
S1131240E025ED02354025435D6010E005224B6941
S11312505D68214C2C401500EDB22E04E025ED0212
S1131260354025435D6002E002006B461A706A4611
S11312701278002A1AD0029A9288002A13D0029A6D
S11312809288092A0FDA029A9288521E4B695D6885
S1131290134C2C401500EDB22E02E025ED00354034
S11312A025435D6002E002006B461A70029A1278D0
S11312B0002A01D0012200E002004B695868102482
S11312C0A0431400E4B2240110252C4004435C60C4
S11312D068460078FEBD0000FFFFF8FFFFFFC7FF70
S11312E0FFF8FFFF0200106A08600120704700B594
S11312F002005068806C03091800C007C00FC0B218
S1131300002804D0FA2080000860012000E00020BA
S113131000BD70B502000878002801D0012400E067
S113132000245368986C1025A8432500EDB22D01C4
S11313301026354005439D64012070BD00B50200B0
S11313405068406C03091800C007C00FC0B20028E1
S113135004D0FA20C0010860012000E0002000BD94
S113136070B502000878002801D0012400E00024B0
S11313705368586C1025A8432500EDB22D011026A2
S1131380354005435D64012070BD0200FA2040022F
S11313900860012070477CB505000E0000200400A1
S11313A0696809680A091100C907C90FC9B2002987
S11313B035D000906868006D000C8007800FC0B2C3
S11313C0002805D002280FD008D3032812D017E034
S11313D069462800FEF71AFF040011E06946280058
S11313E0FEF78EFE04000BE069462800FEF71FFF9F
S11313F0040005E069462800FFF7B0FA0400FFE79F
S11314002000C0B201280AD16868006D000A0107F3
S1131410090F0098C9B2491C01F0AFFC30602000EC
S1131420C0B276BD70B502000878002801D001244E
S113143000E00024536818681025A8432500EDB285
S11314402D011026354005431D60012070BD70B587
S113145004000E0000256068806801090800C007C8
S1131460C00FC0B2002804D031002000FFF72AFCCE
S113147005002800C0B270BD70B5020008780028CD
S113148001D0012400E00024536898681025A84383
S11314902500EDB22D011026354005439D60012045
S11314A070BD70B504000E0000256068C0680109B5
S11314B00800C007C00FC0B2002804D031002000CB
S11314C0FFF700FC05002800C0B270BD70B5020033
S11314D00878002801D0012400E000245368D8686B
S11314E01025A8432500EDB22D01102635400543F3
S11314F0DD60012070BD70B504000E000025606839
S1131500006901090800C007C00FC0B2002804D058
S113151031002000FFF7D6FB05002800C0B270BDE3
S113152070B502000878002801D0012400E00024EE
S1131530536818691025A8432500EDB22D01102623
S1131540354005431D61012070BDF8B505000F004D
S11315500020040000906868C06901090800C00701
S1131560C00FC0B2002801D1002054E068680726EB
S1131570C069000C3040C0B200280BD0022815D03E
S11315800ED304281ED017D3062827D020D307282B
S11315902AD02FE069462800FFF7BEF8040029E0AE
S11315A069462800FEF791FF040023E069462800FD
S11315B0FFF7D4F904001DE069462800FFF7E5FEB3
S11315C0040017E069462800FFF791FE040011E0CB
S11315D069462800FFF7B2FE04000BE069462800C4
S11315E0FFF780FE040005E069462800FFF794F841
S11315F00400FFE72000C0B200280AD06868C06970
S1131600000A06403100C9B2491C009801F0B5FB3C
S113161038602000C0B2F2BDF3B501000120020021
S11316206B461A70002214004D68EE6910239E4325
S113163010232700FFB23F011F403743EF61019E93
S11316407678032E1CD0052E0AD0072E28D00E2E15
S113165066D00F2E44D0102E52D0112E30D06FE011
S113166014004D68EE69AA4F3740BC462600F6B216
S11316703704E026F6023E4067463E43EE6162E0F0
S113168004004D68EE69A24F3740BC462600F6B20E
S11316903704E026F6023E4067463E43EE6152E0E0
S11316A002244D68EE699A4F3740BC462600F6B2D4
S11316B03704E026F6023E4067463E43EE6142E0D0
S11316C003244D68EE69924F3740BC462600F6B2BB
S11316D03704E026F6023E4067463E43EE6132E0C0
S11316E004244D68EE698A4F3740BC462600F6B2A2
S11316F03704E026F6023E4067463E43EE6122E0B0
S113170005244D68EE69824F3740BC462600F6B288
S11317103704E026F6023E4067463E43EE6112E09F
S113172006244D68EE697A4F3740BC462600F6B26F
S11317303704E026F6023E4067463E43EE6102E08F
S113174014006D462C70019CA488002C15D0019CBB
S1131750A488092C11DA019CA488641E4D68EE69E2
S1131760BF4F3740BC462600F6B23702E026F600EB
S11317703E4067463E43EE6102E014006D462C7025
S1131780019C2478002C01D00200FFE74C68E0693A
S11317901025A8431500EDB22D012B400343E3614E
S11317A068460078F6BD70B504000E000025616837
S11317B00120096A09090140C9B2002901D10020A8
S11317C026E06168096A090C8907890FC9B20029F2
S11317D005D002290FD008D3032912D016E0310016
S11317E02000FEF799FF050010E031002000FFF70C
S11317F0B5F805000AE031002000FEF766FE05009A
S113180004E0FA21490231600500FFE72800C0B274
S113181070BDF2B582B00100012002006B461A705F
S113182000226B465A704D682E6A1023DB431E401B
S113183010246F467F783F01274037432F62029E72
S11318407678032E2AD0052E04D0072E13D0112E1D
S113185037D049E06D466A704D682E6AC84F3740EC
S1131860BC466E4676783704C026B6023E406746CC
S11318703E432E623AE005004E680196019E366AA8
S1131880BF4F3740BC462E00F6B23704C026B6021E
S11318903E4067463E43019F3E6227E002254E6874
S11318A00196019E366AB64F3740BC462E00F6B20A
S11318B03704C026B6023E4067463E43019F3E625F
S11318C014E003254E680196019E366AAC4F3740FA
S11318D0BC462E00F6B23704C026B6023E40674628
S11318E03E43019F3E6201E06D462A70029D2D78C1
S11318F0002D01D00200FFE74D68286A0340100064
S1131900C0B2000104401C432C6268460078FEBD4E
S1131910FFFFF8FF70B504000E0000256068806AC0
S113192001090800C007C00FC0B2002801D100207F
S113193027E06068806A000C8007800FC0B200282E
S113194005D002280FD008D3032812D017E03100A5
S11319502000FFF7F3FC050011E031002000FFF741
S1131960C1FC05000BE031002000FFF7C0FC0500BE
S113197005E031002000FFF7BAFC0500FFE728006E
S1131980C0B270BDF2B582B0010000206A4610708A
S113199005004C68A66A1022D243164010232F007B
S11319A0FFB23F011F403743A762029E7678102E94
S11319B011D16C4660704C68A66A714D35406E4614
S11319C076783704C026B6023E402E43A66201252F
S11319D06F463D7031E0029C64780E2C15D10124D1
S11319E025004E680196019EB66A654F3740BC4695
S11319F02E00F6B23704C026B6023E4067463E4388
S1131A00019FBE626F463C7017E0029C64780F2C05
S1131A1013D102244D68AE6A594F3740BC462600A4
S1131A20F6B23704C026B6023E4067463E430196EE
S1131A30019EAE6201266F463E70029C2478002C03
S1131A4001D0012400E004004D68A86A024020008F
S1131A50C0B2000103401343AB6268460078FEBD88
S1131A60FFF8FFFF70B504000E0000256168012037
S1131A70096B090C0140C9B2002905D131002000CD
S1131A80FFF720F905000BE06168096B090C0840B9
S1131A90C0B2012804D131002000FFF776FC050014
S1131AA02800C0B270BDF0B50200002318004C78C5
S1131AB00B2C0CD15468266B564D35401E00F6B2E3
S1131AC037048026760237402F4327630FE04B7894
S1131AD0112B0CD101235468266B4E4D35401E004A
S1131AE0F6B237048026760237402F432763C0B20C
S1131AF0F0BD70B504000E00002561680120496B3B
S1131B00090C0140C9B2002905D131002000FFF7BA
S1131B10D9F805000BE06168496B090C0840C0B2B4
S1131B20012804D131002000FFF72FFC0500280014
S1131B30C0B270BDF0B50200002318004C780B2C25
S1131B400CD15468666B334D35401E00F6B2370431
S1131B508026760237402F4367630FE04B78112BC2
S1131B600CD101235468666B2A4D35401E00F6B231
S1131B7037048026760237402F436763C0B2F0BD36
S1131B80FFFFFCFF70B504000E0000256168012012
S1131B90896B090C0140C9B2002905D1310020002C
S1131BA0FFF790F805000BE06168896B090C0840A9
S1131BB0C0B2012804D131002000FFF7E6FB050084
S1131BC02800C0B270BDF0B50200002318004C78A4
S1131BD00B2C0CD15468A66B0E4D35401E00F6B28A
S1131BE037048026760237402F43A7630FE04B78F3
S1131BF0112B0CD101235468A66B064D35401E00F1
S1131C00F6B237048026760237402F43A763C0B26A
S1131C10F0BD0000FFFFFEFF70B504000E000025BC
S1131C2021680120C96809090140C9B2002905D108
S1131C3031002000FFF746F805000AE02168C96872
S1131C4009090140C9B2012903D1FA2149023160CD
S1131C5005002800C0B270BDF0B5020000231800D2
S1131C604C780B2C0DD11468E5681026B5431E0082
S1131C70F6B2360110273E402E43E66001252800C7
S1131C8012E04B78112B0FD101231C001568EF686B
S1131C901026B743BC462600F6B2360110273E4054
S1131CA067463E43EE601800C0B2F0BD38B505008B
S1131CB00C002869006801090800C007C00FC0B201
S1131CC0002801D1002003E021002800FEF7C6FF10
S1131CD032BD70B502000878002801D0012400E06C
S1131CE00024136918681025A8432500EDB22D01BE
S1131CF01026354005431D60012070BD38B5050030
S1131D000C002869406801090800C007C00FC0B270
S1131D10002801D1002003E021002800FEF7D2FFB3
S1131D2032BD70B502000878002801D0012400E01B
S1131D300024136958681025A8432500EDB22D012D
S1131D401026354005435D60012070BD38B505009F
S1131D500C002869006901090800C007C00FC0B25F
S1131D60002801D1002003E021002800FEF7AAFF8B
S1131D7032BD70B502000878002801D0012400E0CB
S1131D800024136918691025A8432500EDB22D011C
S1131D901026354005431D61012070BD38B505008E
S1131DA00C002869406901090800C007C00FC0B2CF
S1131DB0002801D1002003E021002800FEF782FF63
S1131DC032BD70B502000878002801D0012400E07B
S1131DD00024136958691025A8432500EDB22D018C
S1131DE01026354005435D61012070BD38B50500FE
S1131DF00C002869806901090800C007C00FC0B23F
S1131E00002801D1002003E021002800FEF726FF6E
S1131E1032BD70B502000878002801D0012400E02A
S1131E200024136998691025A8432500EDB22D01FB
S1131E301026354005439D61012070BD38B505006D
S1131E400C002869C06901090800C007C00FC0B2AE
S1131E50002801D1002003E021002800FEF732FF12
S1131E6032BD70B502000878002801D0012400E0DA
S1131E7000241369D8691025A8432500EDB22D016B
S1131E80102635400543DD61012070BD7CB5050099
S1131E900E00002004006968096D0A091100C907D1
S1131EA0C90FC9B2002935D000906868006D000CD4
S1131EB08007800FC0B2002805D002280FD008D3B5
S1131EC0032812D017E069462800FEF79FF90400A2
S1131ED011E069462800FEF713F904000BE0694697
S1131EE02800FEF7A4F9040005E069462800FEF77F
S1131EF035FD0400FFE72000C0B201280AD168685C
S1131F00006D000A0107090F0098C9B2491C00F0CE
S1131F1034FF30602000C0B276BDF3B5010001206B
S1131F2002006B461A70002214004D682E6D1023B7
S1131F309E4310232700FFB23F011F4037432F6504
S1131F40019E7678002E16D0012E04D0022E22D0C7
S1131F50072E30D03FE014004D682E6D8D4F374072
S1131F60BC462600F6B23704C026B6023E40674699
S1131F703E432E6532E004004D682E6D854F374098
S1131F80BC462600F6B23704C026B6023E40674679
S1131F903E432E6522E002244D682E6D7D4F37406E
S1131FA0BC462600F6B23704C026B6023E40674659
S1131FB03E432E6512E003244D682E6D754F374065
S1131FC0BC462600F6B23704C026B6023E40674639
S1131FD03E432E6502E014006D462C70019CA488DB
S1131FE0002C15D0019CA488112C11DA019CA48822
S1131FF0641E4D682E6DAA4F3740BC462600F6B2CB
S11320003702F02636013E4067463E432E6502E025
S113201014006D462C70019C2478002C01D0020021
S1132020FFE74C68206D1025A8431500EDB22D0183
S11320302B400343236568460078F6BD38B5050098
S11320400C006868806D01090800C007C00FC0B2A9
S1132050002801D1002003E021002800FEF732FE11
S113206032BD70B502000878002801D0012400E0D8
S113207000245368986D1025A8432500EDB22D0166
S11320801026354005439D65012070BD70B50500DF
S11320900C0028690126006B00093040C0B20028FA
S11320A001D1002023E02869006B000C8007800F19
S11320B0C0B2002805D002280DD007D303280FD0C2
S11320C013E021002800FEF727FB0FE02100280081
S11320D0FEF7FBF90AE021002800FEF73FFC05E0CB
S11320E021002800FEF718FB00E00020C0B270BDFC
S11320F0FEB5020000206B4618706B4658701369D9
S11321001E6B1024E443264010256F467F783F0160
S11321102F4037431F634E78052E01D103000AE098
S11321204B78032B01D1012305E04B78072B01D118
S1132130022300E0FF231E00F6B2FF2E17D06E46E6
S1132140737016690196019E366B124F3740BC4678
S11321506E4676783704C026B6023E4067463E4354
S11321600296029E019F3E6301266F463E700E78E2
S1132170002E01D0012600E006001769386B0440E8
S11321803000C0B20001054025433D636846007835
S1132190FEBD0000FFFFFCFF70B505000C002869C0
S11321A00126406B00093040C0B2002801D1002054
S11321B023E02869406B000C8007800FC0B2002820
S11321C005D002280DD007D303280FD013E0210037
S11321D02800FEF7A1FA0FE021002800FEF775F9A8
S11321E00AE021002800FEF7B9FB05E021002800E1
S11321F0FEF792FA00E00020C0B270BDFEB5020006
S113220000206B4618706B46587013695E6B10247F
S1132210E443264010256F467F783F012F40374323
S11322205F634E78052E01D103000AE04B78032B3F
S113223001D1012305E04B78072B01D1022300E0F3
S1132240FF231E00F6B2FF2E17D06E467370166978
S11322500196019E766B964F3740BC466E46767863
S11322603704C026B6023E4067463E430296029EAD
S1132270019F7E6301266F463E700E78002E01D0CA
S1132280012600E006001769786B04403000C0B2F4
S11322900001054025437D6368460078FEBD0000CB
S11322A0FFF0FFFF70B505000C0028690126006CE3
S11322B000093040C0B2002801D1002023E0286981
S11322C0006C000C8007800FC0B2002805D00228E3
S11322D00DD007D303280FD013E021002800FEF708
S11322E01BFA0FE021002800FEF7EFF80AE02100B6
S11322F02800FEF733FB05E021002800FEF70CFA66
S113230000E00020C0B270BDFEB5020000206B46A4
S113231018706B46587013691E6C1024E4432640F1
S113232010256F467F783F012F4037431F644E7856
S1132330052E01D103000AE04B78032B01D10123C0
S113234005E04B78072B01D1022300E0FF231E0098
S1132350F6B2FF2E17D06E46737016690196019E71
S1132360366C534F3740BC466E4676783704C026E9
S1132370B6023E4067463E430296029E019F3E647B
S113238001266F463E700E78002E01D0012600E033
S113239006001769386C04403000C0B200010540E3
S11323A025433D6468460078FEBD70B505000C0009
S11323B028690126406C00093040C0B2002801D1D0
S11323C0002023E02869406C000C8007800FC0B215
S11323D0002805D002280DD007D303280FD013E01E
S11323E021002800FEF798F90FE021002800FEF7ED
S11323F06CF80AE021002800FEF7B0FA05E021009D
S11324002800FEF789F900E00020C0B270BDFEB5D7
S1132410020000206B4618706B46587013695E6C9E
S11324201024E443264010256F467F783F012F4057
S113243037435F644E78052E01D103000AE04B78E0
S1132440032B01D1012305E04B78072B01D1022393
S113245000E0FF231E00F6B2FF2E17D06E46737005
S113246016690196019E766C114F3740BC466E4644
S113247076783704C026B6023E4067463E4302964D
S1132480029E019F7E6401266F463E700E78002EE8
S113249001D0012600E006001769786C0440300082
S11324A0C0B20001054025437D6468460078FEBD46
S11324B0FFFFFCFF70B505000C0028690126006EC3
S11324C000093040C0B2002801D1002023E028696F
S11324D0006E000C8007800FC0B2002805D00228CF
S11324E00DD007D303280FD013E021002800FEF7F6
S11324F013F90FE021002800FDF7E7FF0AE02100AF
S11325002800FEF72BFA05E021002800FEF704F965
S113251000E00020C0B270BDFEB5020000206B4692
S113252018706B46587013691E6E1024E4432640DD
S113253010256F467F783F012F4037431F664E7842
S1132540052E01D103000AE04B78032B01D10123AE
S113255005E04B78072B01D1022300E0FF231E0086
S1132560F6B2FF2E17D06E46737016690196019E5F
S1132570366E124F3740BC466E4676783704C02616
S1132580B6023E4067463E430296029E019F3E6667
S113259001266F463E700E78002E01D0012600E021
S11325A006001769386E04403000C0B200010540CF
S11325B025433D6668460078FEBD0000FFFFFCFF32
S11325C038B505000C002869C06E01090800C00771
S11325D0C00FC0B2002801D1002003E02100280070
S11325E0FEF770FB32BD70B502000878002801D0F8
S11325F0012400E000241369D86E1025A8432500A7
S1132600EDB22D01102635400543DD66012070BD75
S113261038B505000C002869006F01090800C007DF
S1132620C00FC0B2002801D1002003E0210028001F
S1132630FEF748FB32BD70B502000878002801D0CF
S1132640012400E000241369186F1025A843250015
S1132650EDB22D011026354005431D67012070BDE4
S113266038B505000C00286980214058010908008C
S1132670C007C00FC0B2002801D1002003E0210030
S11326802800FEF7EBFA32BD70B502000878002886
S113269001D0012300E00023146980202058102574
S11326A0A8431D00EDB22D011026354005438020BE
S11326B02550012070BD38B505000C00286984211F
S11326C0405801090800C007C00FC0B2002801D15A
S11326D0002003E021002800FEF7C0FA32BD70B5E7
S11326E002000878002801D0012300E000231469C7
S11326F0842020581025A8431D00EDB22D0110267A
S11327003540054384202550012070BD38B50500AF
S11327100C0028699421405801090800C007C00F23
S1132720C0B2002801D1002003E021002800FDF7F9
S1132730E7FC32BD70B502000878002801D00123FF
S113274000E000231469942020581025A8431D009C
S1132750EDB22D011026354005439420255001206B
S113276070BD38B505000C0028699C21405801094A
S11327700800C007C00FC0B2002801D1002003E048
S113278021002800FDF753FD32BD70B50200087822
S1132790002801D0012300E0002314699C20205864
S11327A01025A8431D00EDB22D0110263540054328
S11327B09C202550012070BD0200506A0860012051
S11327C070470200906A0860012070470200D06AD6
S11327D008600120704770B505000C0001262869C7
S11327E0A0214058000C4007400FC0B200280BD075
S11327F0022813D00DD304281AD014D3062821D0CC
S11328001BD307281ED022E021002800FFF7D4FFA5
S11328101EE021002800FFF7D4FF19E02100280062
S1132820FFF7D4FF14E021002800FEF707F80FE0BB
S113283021002800FDF7DCFE0AE021002800FEF755
S11328401DF905E021002800FDF7F8FF00E0002055
S1132850C0B270BDF0B50200012318004C78042CFE
S113286049D0062C37D0082C55D0302C04D0312C2C
S113287012D0322C1FD05EE000231469A0256659C3
S1132880AD4D35401E00F6B23704E026F6023E4058
S11328902E43A025665150E01469A0256659A64D23
S11328A035401E00F6B23704E026F6023E402E43C1
S11328B0A025665141E002231469A02566599E4D66
S11328C035401E00F6B23704E026F6023E402E43A1
S11328D0A025665131E003231469A0256659964D5D
S11328E035401E00F6B23704E026F6023E402E4381
S11328F0A025665121E004231469A02566598E4D54
S113290035401E00F6B23704E026F6023E402E4360
S1132910A025665111E005231469A0256659864D4A
S113292035401E00F6B23704E026F6023E402E4340
S1132930A025665101E000231800C0B2F0BD70B5B7
S113294005000C0001262869A4214058000C40070A
S1132950400FC0B200280BD0022813D00DD3042896
S11329601AD014D3062821D01BD307281ED022E066
S113297021002800FFF720FF1EE021002800FFF7B8
S113298020FF19E021002800FFF720FF14E02100B8
S11329902800FDF753FF0FE021002800FDF728FE73
S11329A00AE021002800FEF769F805E0210028006C
S11329B0FDF744FF00E00020C0B270BDF0B5020096
S11329C0012318004C78042C49D0062C37D0082C4D
S11329D055D0302C04D0312C12D0322C1FD05EE0D4
S11329E000231469A4256659534D35401E00F6B2E0
S11329F03704E026F6023E402E43A425665150E0FB
S1132A001469A42566594C4D35401E00F6B23704AE
S1132A10E026F6023E402E43A425665141E00223FF
S1132A201469A4256659444D35401E00F6B2370496
S1132A30E026F6023E402E43A425665131E00323EE
S1132A401469A42566593C4D35401E00F6B237047E
S1132A50E026F6023E402E43A425665121E00423DD
S1132A601469A4256659344D35401E00F6B2370466
S1132A70E026F6023E402E43A425665111E00523CC
S1132A801469A42566592C4D35401E00F6B237044E
S1132A90E026F6023E402E43A425665101E00023C1
S1132AA01800C0B2F0BD70B505000C00012006008E
S1132AB02969C0228958090C0840C0B2002802D0F4
S1132AC0012805D009E021002800FEF737FC05E0C5
S1132AD021002800FEF706FC00E00020C0B270BD13
S1132AE0F0B50200012318004C780E2C11D0102CE4
S1132AF01ED100231469C02566598E4D35401E0031
S1132B00F6B2360480277F023E402E43C02566512C
S1132B1010E01469C0256659864D35401E00F6B292
S1132B20360480277F023E402E43C025665101E0D3
S1132B3000231800C0B2F0BDFFFFF8FF70B5050018
S1132B400C00012006002969C4228958090C084098
S1132B50C0B2002802D0012805D009E021002800D5
S1132B60FEF7ECFB05E021002800FEF7BBFB00E0CC
S1132B700020C0B270BDF0B50200012318004C78EB
S1132B800E2C11D0102C1ED100231469C4256659B3
S1132B90684D35401E00F6B2360480277F023E4061
S1132BA02E43C425665110E01469C4256659614D4D
S1132BB035401E00F6B2360480277F023E402E4385
S1132BC0C425665101E000231800C0B2F0BD38B539
S1132BD005000C002869CC21405801090800C007F1
S1132BE0C00FC0B2002801D1002003E0210028005A
S1132BF0FEF734F832BD70B502000878002801D021
S1132C00012300E000231469CC2020581025A84398
S1132C101D00EDB22D01102635400543CC20255072
S1132C20012070BDFEB50899099A0A9B0B9C009D72
S1132C300560019D4560029D8560C160026143613C
S1132C40256885616568C561A568056200252E0053
S1132C502E00F6B2032E0BD22E00F6B2B600A61941
S1132C60F6682F00FFB2BF00C7197E626D1CEFE744
S1132C70F7BDF8B506000C0017002000C0B23828D4
S1132C8001DB002011E000252B4A2000C0B2C00067
S1132C901058002807D0390030002300DBB2DB00D5
S1132CA0D258904705002800C0B2F2BDF4B588B0F0
S1132CB004000F003800C0B2382801DB002037E0E0
S1132CC000252E001C4A3800C0B2C000101840680D
S1132CD000282BD019480790606806900798069939
S1132CE08023C85016480590A0680490059804995C
S1132CF00866144803902068029003980299802380
S1132D00C850089920003B00DBB2DB00D21852689F
S1132D1090470600019560680199802281500095D2
S1132D20A168009A0A6622688023D5503000C0B298
S1132D3009B0F0BDFFFFFEFFECAE00005245535555
S1132D40202096194B4D4352F446002804D449429E
S1132D5000F013F8404260474042002905D45FD098
S1132D6000F00BF8404249426047494200F005F840
S1132D704942604703460B43E6D40022030A8B42D0
S1132D800BD203098B4219D243088B422ED2411A2B
S1132D9000D20146524110467047FF2209023FD03B
S1132DA012068B4205D3121209028B4201D312126E
S1132DB0090203098B4219D300E0090AC3098B42B3
S1132DC001D3CB01C01A524183098B4201D38B0139
S1132DD0C01A524143098B4201D34B01C01A5241DC
S1132DE003098B4201D30B01C01A5241C3088B4221
S1132DF001D3CB00C01A524183088B4201D38B000C
S1132E00C01A524143088B4201D34B00C01A5241AD
S1132E10884200D3401A5241CFD20146104670472F
S1132E2008B500F001F808BD7047FEE700B50100E1
S1132E3000200A00D2B2002A05D0022A09D005D304
S1132E40032A09D00AE01022100007E0182210001B
S1132E5004E02822100001E048221000C0B200BDA6
S1132E60F8B505000C00286806008036002768467F
S1132E7007703800C0B2FFF7D9FF0100C9B2890852
S1132E800800C0B2220092B2504380003018F2BD54
S1132E9000B5010000200A00D2B2002A082A0ED987
S1132EA0093A0ED0521E0FD0521E10D0521E11D00D
S1132EB0521E12D0521E13D0521E14D016E0080017
S1132EC014E00C22100011E0102210000EE0142275
S1132ED010000BE01822100008E02022100005E08A
S1132EE03022100002E040221000FFE7C0B200BD13
S1132EF0F8B505000C000020694648706946087062
S1132F00210089B22800FFF7ABFF06003068000CEF
S1132F1007073F0F3800C0B2FFF7BAFFC0B2F2BDD7
S1132F2070B500231400E4B2002C0CD00468C02552
S1132F30ED03254305604468640F6407CD00ED0884
S1132F40254345600BE00468C74D2540056044688F
S1132F50C64E26408C04C64D25403543456070BDA1
S1132F6010B40268C34B1340036002680B00DBB269
S1132F701B04F02424031C401443046010BC704759
S1132F8000B502685200520802600268BA4B13404E
S1132F9003600A00D2B2002A09D0026880231B060B
S1132FA01343036002688023DB051343036000BD01
S1132FB000B50A00D2B2002A06D10268AF4B134012
S1132FC00360026802600CE00A00D2B2012A08D150
S1132FD00268AA4B1340036002688023DB04134396
S1132FE0036000BD30B50268803200231D001C0060
S1132FF0057EED01AC4205D2A500551929000B60F0
S1133000641CF5E730BDF8B49D4982688023D15033
S113301001234468256D2026B5431E00F6B27601CF
S113302020273E402E430096009D25650025866896
S11330308027F551F1BC7047F8B491498268802328
S1133040D15001234468256D1026B5431E00F6B205
S1133050360110273E402E430096009D256500252D
S113306086688027F551F1BC7047F0B48549C26881
S1133070116601230469E6691025AE431D00EDB213
S11330802D0110273D403543E5610026C7683E66A3
S1133090F0BC7047F2B40599069C079D089E3778EA
S11330A00776009F076042608360C16004614561E8
S11330B0F1BC704730B500221100826002614261A8
S11330C08261C260C26142628262C26202620123A0
S11330D003701300C370130003710023DB434363C5
S11330E08363C363036414004425445514004525D5
S11330F044551400C8254455082446254455140055
S11331002100C9B2202906DA2100C9B28900411878
S11331108B64641CF4E7110041701100817011008C
S11331203023C1541100C923C1541100CA23C1540E
S11331301100CB23C1541100D523C1541100D42351
S1133140C1541100D623C1541100D723C154110016
S1133150CC23C154D021425030BDF0B5002421000D
S113316002681368444D1D400B00DBB29B078026A8
S1133170F60533402B43136005682E68424F3740F1
S1133180BC462600F6B2360780277F053E406746D8
S11331903E432E60016809680A0E1100C907C90F71
S11331A0C9B20029F6D1F0BDF8B5040020680125A4
S11331B00068000D2840C0B2002814D00020216807
S11331C00A68520052080300DBB2DB0713430B60AA
S11331D020680068000D2840C0B2002803D02000F9
S11331E0FFF72AFFF4E7280021680B68274A1A40F2
S11331F00300DBB25B068026B604334013430B6046
S113320020680068400E2840C0B20028F8D1684603
S1133210057020680168184A0A40694609788907D8
S11332208023DB051940114301602A0023681E68CE
S1133230154F3740BC461600F6B2360780277F0587
S11332403E4067463E431E6020680068000E2840EA
S1133250C0B20028F8D020680068C00E2840C0B270
S11332600028F1D0F1BD0000FFFF9FFFFFFF03E046
S11332700000FC1FFFFFF0FFFFFFFFBFFFFFFFF099
S11332805245535520209619FFFFFFEFFFFFFFFD26
S1133290F8B594B007000C0016003100C9B289B229
S11332A03800FFF7DDFD0500227A61682800FFF78A
S11332B037FEA17A2800FFF753FEE17A2800FFF7D2
S11332C05FFE617A2800FFF773FE207B002805D09B
S11332D06846067101A9380000F0BDFC607A012837
S11332E00AD1206969460E7039686A4612789200DC
S11332F08A1888231B01D05015B0F0BDF0B58DB0ED
S113330005000E00002069464870002069460870D8
S11333102800FFF778FE3078002802D12800FFF754
S1133320A4FE012029680A68520052080300DBB297
S1133330DB0713430B6028680068010D0800C00711
S1133340C00FC0B20028F6D03078694648712868AA
S1133350029002984068CE49014068464079400393
S11333608022920110400843059005980299486014
S11333702800FFF719FF0120694608712F68396892
S1133380E548084069460979C905802212041140BC
S1133390014304910498386001206946C8702C6880
S11333A0616BDE4808406946C978090780225205E6
S11333B0114001430391039860632800FFF712FE54
S11333C03020305CFFF732FD6946887068468078AB
S11333D0002809D08020800069468978FFF7CDFC59
S11333E0297E4843694648706846407869460871B2
S11333F028680690069800687F2188436946097901
S11334004906490E01430C910C9806990860012065
S11334106946C870286805900598006D400040080A
S11334206946C978C90701430B910B98059908654A
S1133430BB48B16809186A46D18129680491049986
S11334400A6DB84911406A46D2895205B64B1340F9
S11334500B430A930A99049A1165F16809186A469C
S1133460918129680B6DB14A1A406B469B891B04F4
S1133470F82464031C4014430994099A0A653269C8
S113348012186B465A812A68146DA94B23406C4666
S11334906489A702FC2424023C401C430894089B32
S11334A0136573691B186C4623812B681C6DA14F2F
S11334B02740BC466C4624896701F824A4003C409C
S11334C067463C430794079C1C65B46920186C4606
S11334D0E0802868046D1F27BC436F46FF88FF0601
S11334E0FF0E27430765F478002C6ED0012069464F
S11334F0887128680268DF4911406A469279520748
S113350080239B051A400A4306920699016031798B
S11335106A46517129680B68D74A1A406B465B7931
S1133520DB0380242402234013430593059A0A6095
S1133530326C04922A680392049A039B9A6444228C
S1133540B25C6B461A712A681468CC4B23406C46F3
S113355024792702C024A4003C401C430294029B0B
S113356013604523F35C6C46E3702B685C6BC44FBB
S11335702740BC466C46E4782706F02424053C40EA
S113358067463C435C63C827F75D012F3BD10020AD
S113359069460870684600784621715C884232D2D8
S11335A06846007880003018806C694609782A687B
S11335B00B00DBB29B00D3188824240118516B46FE
S11335C01B785B1C6C462370E4E7002029680B68B9
S11335D0A84A1A400300DBB25B078024A4052340F9
S11335E013430193019A0A6000222B681C68A24FBE
S11335F02740BC461400E4B2E40380273F023C4069
S113360067463C431C60706B039028680399016112
S1133610B16B02912968029A4A61F26B01922A689D
S1133620019B9361C823F35C6C46E3702B681C68B0
S1133630944F2740BC466C46E478240480277F02DC
S11336403C4067463C431C60C927F75D002F21D0EE
S1133650002029680B688C4A1A400300DBB25B0423
S11336608024A402234013430193019A0A60012297
S11336702B685C68854F2740BC461400E4B22403E1
S113368080277F013C4067463C435C6020E000BFEC
S1133690FFDFFFFF012029680B687B4A1A40030003
S11336A0DBB25B048024A402234013430193019AF8
S11336B00A6000222B685C68744F2740BC461400E3
S11336C0E4B2240380277F013C4067463C435C60AE
S11336D0D420305C00282FD00122100029680C6807
S11336E06B4B23400400E4B2A4058027FF033C4055
S11336F01C430194019B0B606B46DA702A681468C2
S1133700644B23406C46E478A7068024E4042740F5
S11337101F4317602EE000BFFFFF7FFFFFFFFFEF97
S1133720FFFF0000FFFF1F800000E07FFFFFE0FFBE
S1133730FF03FFFF1FFCFFFF0022100029680C6835
S1133740534B23400400E4B2A4058027FF033C400C
S11337501C430194019B0B602B681C684D4F274050
S1133760BC461400E4B2A4068027FF043C4067462C
S11337703C431C60D520305C6946087128680268A7
S1133780424911406A461279120380235B011A40B0
S11337900A43049204990160D621715C6A46D1708F
S11337A029684B68344A1A406B46DB78DB03802473
S11337B02402234013430393039A4A60D722B25C42
S11337C02B685C68344F2740BC461400E4B2A40361
S11337D08027FF013C4067463C430294029C5C60A6
S11337E000273800CC21715CC0B288422DD2002061
S11337F0D02171583A00D2B214235A438C5A220071
S113380092B2D02030583900C9B214235943435AD4
S1133810D020305884463900C9B214204143604650
S113382040184088181882420DDA2200D2B2D02003
S113383030583900C9B21423594341182800FFF7FE
S113384027FD641CDBE77F1CCBE7280000F087F929
S11338502800FFF782FC002029680B680F4A1A40F1
S11338600300DBB2DC0580231B041C4014430C6002
S11338700DB0F0BDFFFFFFDFFF7FFFFFFFFCFFFF89
S1133880FFFFFFF0FFFFFEFFFFFFFDFFFFEFFFFF66
S1133890FFFFBFFFFFFFFFFBFFBFFFFFFFFF7FFF38
S11338A038B504000D00297889B22000FFF7D8FA52
S11338B00168C02212050A43026031BDF1B50C0053
S11338C0217889B20098FFF7CBFA050008352178F2
S11338D089B20098FFF70CFB00210B000A001300CB
S11338E0DBB2834238D203231E00324209D129605D
S11338F02B681600F6B2A619367A36061E432E60D9
S113390028E01600F6B21E40012E08D12B681600DE
S1133910F6B2A619367A36041E432E601AE0160053
S1133920F6B21E40022E08D12B681600F6B2A61974
S1133930367A36021E432E600CE01600F6B233408F
S1133940032B07D12B681600F6B2A619367A1E434C
S11339502E602D1D521CC2E7F1BDF8B506000C0007
S1133960217889B23000FFF77BFA05002868000C43
S11339700007000FFFF78CFA482160542868400DB7
S11339800100C907C90F68460170281D69460978F6
S1133990002904D00168C900C908616004E0016815
S11339A0890C4905490D6160051D217889B23000F3
S11339B0FFF79EFA00210A000A000300D2B2DBB22C
S11339C09A422AD203221300194206D12A68120EFF
S11339D00B00DBB2E3181A721DE00B00DBB21340DC
S11339E0012B06D12A68120C0B00DBB2E3181A7201
S11339F011E00B00DBB21A40022A06D12A68120A2F
S1133A000B00DBB2E3181A7205E02A680B00DBB284
S1133A10E3181A722D1D491CCEE732689268F1BD75
S1133A20F0B500252E000A78D206D20E0124230018
S1133A3093400F78402F12DB1C0002260568002EED
S1133A400AD0022E04D005D3032E07D12C6705E03B
S1133A506C6703E0EC6201E02C63FFE725E00E787D
S1133A60202E11DB1D000668002C0AD0022C04D085
S1133A7005D3032C07D1356705E0756703E0F562CC
S1133A8001E03563FFE710E01C000668002D0AD052
S1133A90022D04D005D3032D07D1346705E07467E4
S1133AA003E0F46201E03463FFE7F0BDF0B5030026
S1133AB0002215000878C406E40E01200600A64082
S1133AC00F78402F16DB02201D6800280DD0022835
S1133AD005D007D303280BD12F6F3A0008E06F6F8E
S1133AE03A0005E0EF6A3A0002E02F6B3A00FFE784
S1133AF032402EE00D78202D15DB1D6800280DD0F6
S1133B00022805D007D303280BD12F6F3A0008E011
S1133B106F6F3A0005E0EF6A3A0002E02F6B3A005B
S1133B20FFE7324015E010001D6800280DD0022880
S1133B3005D007D303280BD12F6F3A0008E06F6F2D
S1133B403A0005E0EF6A3A0002E02F6B3A00FFE723
S1133B503240002A01D0012000E00020F0BDF0B581
S1133B60017E032937D10021C9430D0002270668CD
S1133B70002F0AD0022F04D005D3032F07D13567B5
S1133B8005E0756703E0F56201E03563FFE70A00CD
S1133B9001230468002B0AD0022B04D005D3032B85
S1133BA007D1226705E0626703E0E26201E0226375
S1133BB0FFE700260568002E0AD0022E04D005D3A4
S1133BC0032E07D1296705E0696703E0E96201E094
S1133BD02963FFE73EE0017E022925D10021C94384
S1133BE00A0001250368002D0AD0022D04D005D354
S1133BF0032D07D11A6705E05A6703E0DA6201E092
S1133C001A63FFE700260468002E0AD0022E04D0AF
S1133C1005D3032E07D1216705E0616703E0E16264
S1133C2001E02163FFE715E0017E012912D10021A3
S1133C30C94300230268002B0AD0022B04D005D309
S1133C40032B07D1116705E0516703E0D16201E05E
S1133C501163FFE7F0BDF0B500231E000A78D40617
S1133C60E40E01221500A5400F78402F1ADB2A002C
S1133C7002230668002B10D0022B06D009D3032B95
S1133C800FD1B76E1743B7660BE0F76E1743F766AD
S1133C9007E0776A1743776203E0B76A1743B762AE
S1133CA0FFE735E00E78202E19DB2B000668002A8A
S1133CB010D0022A06D009D3032A0FD1B76E1F43AE
S1133CC0B7660BE0F76E1F43F76607E0776A1F439A
S1133CD0776203E0B76A1F43B762FFE718E02A0080
S1133CE00668002B10D0022B06D009D3032B0FD16A
S1133CF0B76E1743B7660BE0F76E1743F76607E036
S1133D00776A1743776203E0B76A1743B762FFE73E
S1133D10F0BDFFB591B00025012009900120089065
S1133D20082001900321049102220592142210928A
S1133D30834A0F92FA2292050E921BAA1278002A45
S1133D400DD1804A0D925E2202920C911F2107919F
S1133D500299079A8918491C0B910A900CE0794A38
S1133D600D92262202920C91072107910299079A3B
S1133D708918491C0B910A90139800F0EDF804007F
S1133D8001260D98B04259DB129800F0E5F80500C1
S1133D90300000F0F1F80100280000F0F8F8050008
S1133DA0139800F0D9F80100280000F0F0F800F0B2
S1133DB041F900900098002803D000980A9988429D
S1133DC000DA3BE0009800F0D7F80100280000F08A
S1133DD0DEF80700139800F0BFF80100380000F087
S1133DE07EF98021090400F0D3F908D8139800F073
S1133DF0B3F80100380000F072F9020006E01398ED
S1133E0000F0AAF8390000F06AF902000B98009952
S1133E10884211DB2000110000F0BAF90CD8099691
S1133E2000980190140010980099884204DB100057
S1133E300F9900F0C1F901D3761CA2E714A80088F9
S1133E4000F08AF80E9900F0CAF9039001980299DB
S1133E50884201DA01980290029C0C98844225DB86
S1133E602000401C384948430199FEF783FF0500B0
S1133E7014A80088281A012803DB14A800882F1A24
S1133E8002E014A80088471B14A8008885420DDBB3
S1133E90380000F071F8039900F08EF904D204940C
S1133EA0380000F069F80390641ED6E7019804997D
S1133EB0401A401E05902548039001250598A84204
S1133EC021DB214868430199FEF754FF07001AA833
S1133ED00088381A012804DB1AA80088381A0690CA
S1133EE003E01AA80088C01B0690069800F044F866
S1133EF0039900F061F904D20895069800F03CF8A3
S1133F0003906D1CDAE7099811990860049800F091
S1133F10CFF90FA20CCA00F0D5F900F095FA119967
S1133F208860049811998968401A1199C8600598A5
S1133F301199086108981199486015B0F0BD000006
S1133F40CDCCCC3DFF0300001027000000401C46F0
S1133F50333333333333E33F9D2102000AD002D499
S1133F60491E9218FCD5C905100A1206524100D305
S1133F70012A4841704700009D210200EED55242BB
S1133F80F446FFF7EBFF0122D2071043604730B439
S1133F9005004D400122D20715404B180418240E89
S1133FA025D01B0E2CD0FF2C31D0FF2B34D0E41A9B
S1133FB0000209021043114343084808D10D1B1A9B
S1133FC002D2641EDB181B18DB18834200D31B1AB1
S1133FD04941F9D37F3423DDFF2C05DAE405480891
S1133FE06041284330BC7047FF20C005F9E7280032
S1133FF01B0E03D0FF2BF5D14902F3D0D043F1E7D8
S1134000FF2C01D14002F9D1FF20C005E9E74002AD
S1134010F4D1FF2BF8D1F1E728004902E2D0EDE713
S11340200B0200202442DCD15B129B1CD9D9D80599
S1134030D7E7FEE70122D2070118090E7F3910D411
S113404049421F310FD4001805D2C0011043C840A3
S113405000D5D0437047C0011043C84005D4404246
S11340607047002070470042F3D5100070470122CA
S1134070D20703004B402ED4431A01D2C01AC918E8
S113408030B44B180418240E1B0E22D0FF2C20D061
S1134090E31A182B1DDC09021143C40D641E00022F
S11340A0104394461925ED1A0A00AA40D940451830
S11340B001D36D08A41CE405D209280A2D062A435D
S11340C06546AA41604103181B0EFF2B01D3C00DA6
S11340D0C00530BC7047514006E05140CCE7012296
S11340E0D20703004B40F8D4431A03D2C01AC918AC
S11340F05040514030B44B18090211430418240EA7
S11341001B0E40D0FF2C3AD025009D410BD31ED866
S1134110C50D4002401A0BD3ED050100400AC90544
S113412091416841D5E7C50D40024918401AD0D0E5
S113413001214008491C0018FCD58C4204D36D1A97
S1134140000AED054019C4E7E8051040C1E7182D41
S1134150BFDCAC1C0D00E140E5414D40012D49415F
S1134160C40D00021043451A01D46D199543641E11
S1134170E405280A2D069541604130BC7047FF2BA9
S1134180A7D1D843A5E72442A3D10020A1E7FEE7A5
S11341900CB4012212060318DA4207D84B18DA428B
S11341A004D802000A43921802D281420CBC704720
S11341B0FCD088420CBC70470CB4012212060318D0
S11341C0DA4207D84B18DA4204D802000A4392189C
S11341D002D288420CBC7047FCD08142FAE730B46A
S11341E005004D400122D20715404B180418240E37
S11341F02ED01B0E32D0FF2C34D0FF2B3AD0E41833
S11342000002090210431143000A090A9446C2B28B
S11342104A43000AC3B24B43000A4843110A5B18DD
S11342201A43D2B2190A091801D44918641E080A9B
S11342307F3C23DBFE2C08DAE405090611436346C0
S113424099416041284330BC7047FF20C005F9E71D
S113425028001B0EFF2BF6D1D043F4E72800FF2CD7
S1134260F1D1F9E74002F7D1FF2B01D14902F3D193
S1134270E005E7E7D8054902E4D0EDE74302002072
S1134280641CDFD15B129B1CDCD9D805DAE7FEE79E
S1134290010042221201D21E004207D002D4521E53
S11342A00018FCD5C10A40051205891870470000A2
S11342B00100EED54042F446FFF7EBFF0122D2079E
S11342C011436047F0B50E005E400125ED072E4016
S11342D0B446AE0ADF184C18F44208D2F7420ED2A4
S11342E0640D01D07F0D12D100206146F0BD05D1CF
S11342F0F74201D87F0D05D10020C143F0BDFBD1A9
S1134300640DF9D00020C143490549088FE0E41940
S1134310C902DB0229432B43DB0A460DC0023143A9
S11343208E4630B487B295B27D432E0CADB2140CD8
S11343307C43A419260C240425439CB27C43A41971
S1134340190C7943270CC919A4B20F043C43090C76
S1134350000C97B247432E0CBE193543ADB2170C6F
S11343604743360CBF19A6B2BF193E043543240C8B
S11343703E0C36199FB24743BF19BCB23E0C891993
S11343801F0C47437F183E043443390C704680B2F7
S113439097B247432E0CBE193543ADB2170C4743B1
S11343A0360CBF19A6B2BF193E043543240C3E0C8B
S11343B036199FB24743BF19BCB23E0C89191F0C72
S11343C047437F183E043443390C77463F0C90B280
S11343D078432E0C80190604ADB22E43050CA0B20E
S11343E02D18120C7A435019020C80B2240CA41814
S11343F09AB27A43121914042043120C89181B0C24
S11344007B43C91830BCEF0A394203D1B619404185
S11344104941641E6F12BF0DE41B0BDBFF19BC4244
S113442011DA240500274208AE417841614166460D
S11344303143F0BD641C05D1401C6141CF0201D35E
S11344404908F4E750E75DE74A1812D2400DC90263
S113445008430121C9070843520D40210901521A9A
S1134460521C06D452421F3201D4D0407047C017A8
S11344707047002070470000F8B59CB00500002686
S11344803700300069460870029601963400300007
S113449069468870402200210CA800F00DFE04A893
S11344A0D349202200F012FE082069464870FF20FC
S11344B0801C0390300001006A465278C9B29142D0
S11344C00FD20021C9430CAA0300DBB2DB00D15098
S11344D031000CAA0300DBB2DB00D2189180401C2F
S11344E0E9E73700380069464978C0B288424BD2C0
S11344F0022004000398210089B288423ED3286830
S113450004A93A00D2B292008958FEF736FC210081
S113451089B2FEF732FC019001986968884213D190
S11345200CA83900C9B2C90041188C803900C9B23D
S1134530C900401887710CA83900C9B2C900465097
S113454001206946887019E001986968884213D28D
S11345500CA83900C9B2C90041188C803900C9B20D
S1134560C9004018877168680199401A0CA93A007B
S1134570D2B2D200885001E0641CBBE76846807860
S1134580002801D17F1CADE7684606700CA8694677
S11345900978C900405802900126300069464978DC
S11345A0C0B2884211D20CA83100C9B2C900405827
S11345B00299884207D20CA83100C9B2C9004058F8
S11345C0029068460670761CE7E70CA869460978ED
S11345D0C90041188988022917DA286804A96A469B
S11345E0527892008918091F0968FEF7C6FB0399DF
S11345F0FEF7C3FB019068464078401EA86003980C
S1134600801EE8600198286114E069460978C900B1
S113461041188979A96069460978C90040188088D9
S1134620801EE86068680CA96A461278D20089582E
S1134630401A28611DB0F0BDF8B58AB004000D0021
S113464000200090070002902000006E00900021DE
S1134650684600F0F4FC0021684600F0E1FC697B48
S1134660684600F0A3FC697A684600F075FCA97AF4
S1134670684600F068FC686806902868059005A8FC
S1134680FFF7FAFE07986946087108980290029E9F
S113469003940398006CFF2188433100C9B201439D
S11346A0049104980399086468460179684600F007
S11346B061FCE989491E89B2684600F0F3FCA87BD5
S11346C0800604D5E97E684600F07EFC03E0002104
S11346D0684600F079FCE97A684600F059FC687D88
S11346E0002805D0022829D010D303283ED04BE05F
S11346F00021684600F0B2FCE97F684600F090FCB7
S11347002020295C684600F09AFC4AE001216846B2
S113471000F086FC0021684600F091FC287C00280B
S113472004D10021684600F099FC06E0287C0128A9
S113473003D10121684600F091FC32E0287C002876
S113474004D10021684600F089FC06E0287C012899
S113475003D10121684600F081FC0121684600F084
S11347605FFC0021684600F06AFC1AE000216846FC
S113477000F074FCE97F684600F052FC2020295CBC
S1134780684600F05CFC0CE00021684600F066FC22
S1134790E97F684600F044FC2020295C684600F06C
S11347A04EFC009820660BB0F0BDF8B50A7A6B4653
S11347B01A700200536A6C462478012C03D1012438
S11347C01C43546202E05C08640054620C7BCD7AA2
S11347D0AC4005006E6ACB4F3740BC462600F6B2AB
S11347E03702F02636013E4067463E436E62F1BD15
S11347F030BC0000F6B588B0099909780200D66982
S11348000B00DBB2012B03D101233343D36102E05C
S113481073085B00D361099B5B780400E5691F00A2
S1134820FFB2012F03D102212943E16103E02900F2
S113483002229143E161099989780200566A0F00C6
S1134840FFB2012F03D108233343536203E0330043
S11348500824A3435362099BDB780400256A1F00E4
S1134860FFB2012F04D1802149002943216202E0D3
S1134870A54929402162009000210E000122009FD9
S11348807F6A1740002F01D013001E00F6B2002EDD
S11348900FD1099B5B790400656A1E00F6B2012EF4
S11348A003D104262E43666203E02E000427BE4390
S11348B06662099BDB796C46237005002E696B46A2
S11348C01B78012B03D1042333432B6103E0330012
S11348D00424A3432B61099B9B796C462371030039
S11348E01C696F463F79012F03D1082525431D61BB
S11348F003E025000826B5431D61089D6D786E46CA
S1134900F5700490049D2E6C804D35406E46F6780B
S113491036022E430796079D049E3564089DAD78A4
S11349206E46B5700390039D2E6C794D35406E46EE
S1134930B67836042E430696069D039E3564089D7C
S1134940ED786E4675700290029D2D6C2D022D0A35
S11349506E46767836062E430596059D029E35648E
S1134960089D2D796E46357005006F6A7026B74331
S1134970BC466E463678370170263E4067463E4355
S11349806E62089F7F79002F05D0022F39D024D37F
S1134990032F4AD06DE0089B9B79002B00D10A00BD
S11349A003005C6A1500EDB2002D04D08025ED04EF
S11349B025435D6202E0574D25405D6205006E6A45
S11349C0554F3740BC460E00F6B23706C026B60433
S11349D03E4067463E436E626CE013000400616A29
S11349E04D4D0D401900C9B20E06C0218904314055
S11349F02943616205006E6A8027FF0437436F62B2
S1134A0058E002230400616A434D0D401900C9B205
S1134A100E06C021890431402943616205006E6A93
S1134A208027FF0437436F6244E0089B9B79002B87
S1134A3001D01100FFE70200536A0C00E4B2002C1D
S1134A4004D08024E4041C43546202E0314C1C4032
S1134A505462032405006E6A2F4F3740BC4626007B
S1134A60F6B23706C026B6043E4067463E436E6241
S1134A7020E0089B9B79002B00D10A0003005C6AAC
S1134A801500EDB2002D04D08025ED0425435D62B0
S1134A9002E0204D25405D6205006E6A1E4F3740DE
S1134AA0BC460E00F6B23706C026B6043E40674642
S1134AB03E436E620AB0F0BD8149016081494160A4
S1134AC001220272002141728172C1720173427328
S1134AD00822C281C175017641768176C17601775B
S1134AE04177C177202281548177022202740A22FD
S1134AF01300437413008374C27401754175817586
S1134B0070470000FFF0FFFFFFFEFFFFFF00FFFF05
S1134B10FFFF00FFFFFFFFFBFFFFFFFCF0B587B0C7
S1134B2004000D0000206946487020680290029835
S1134B30006906900698012188430299086120685B
S1134B40019001980069059005988021490001436E
S1134B5001980161276838690490049880218900CC
S1134B600143396100BF00BF00BF29002068FFF77F
S1134B701CFE2A001732290010312068FFF73AFE84
S1134B80012001006A461170266831690391039976
S1134B900843306129002068FFF74EFD07B0F0BDDF
S1134BA0F2B482B00299016001680A690192019A23
S1134BB080235B0013430B61026813690093009B1D
S1134BC08024A4001C43146101230468256902267F
S1134BD02E43266100BF00BF00BF002607683E6168
S1134BE0F7BC7047F0B503000022100014000D005C
S1134BF06D1E17D06D1E1DD0FE3D24D0802676007C
S1134C00AD1B29D08026B600AD1B2ED08026F60021
S1134C10AD1B33D080263601AD1B38D08B4EAD1B77
S1134C203ED046E01D686F693E00F607F60FF6B207
S1134C3034003EE01D686E6977083E00F607F60F03
S1134C40F6B2340035E01D686E69370A3E00F60797
S1134C50F60FF6B234002CE01D686E69770A3E0048
S1134C60F607F60FF6B2340023E01D686E69B70A42
S1134C703E00F607F60FF6B234001AE01D686E69BE
S1134C80F70A3E00F607F60FF6B2340011E01D688D
S1134C906E69370B3E00F607F60FF6B2340008E0F3
S1134CA01D686E69370E3E00F607F60FF6B2340043
S1134CB0FFE7002C01D001221000C0B2F0BD0000BB
S1134CC000B4C40440420F00FFB583B0012069461C
S1134CD0087000242000039909682200CB6DDB06CC
S1134CE0DB0E1025EB1A6D466B706B465B786D46D8
S1134CF0AD8A9BB2AB4200D2A2E001942500200011
S1134D006946488003980068006E0190002101A85C
S1134D1000F078F9012101A800F065F9002101A84B
S1134D2000F08DF9002101A800F07AF96846007CB2
S1134D30C100491E89B201A800F0B4F90198039991
S1134D4009680866260030006946898A80B288426C
S1134D5069D203980168220001204F6903003B4097
S1134D60DBB2002B06D16D1C39498D42F1D32100F1
S1134D706A4611706946097C012907D106993200F7
S1134D8092B2895C039A1268516614E06946097C00
S1134D90022908D10699320092B25200895A039A24
S1134DA01268516607E00699320092B2920089585F
S1134DB0039A1268516625000399096822000B6F53
S1134DC05B080340002B01D003001A00D2B2002A72
S1134DD006D06D1C1E498D42EED320006946087032
S1134DE06846007C012807D103980068406F0C993D
S1134DF0320092B2885414E06846007C022808D13C
S1134E0003980068406F0C99320092B252008852A5
S1134E1007E003980068406F0C99320092B2920048
S1134E208850761C8FE7002101A800F0EBF80021E0
S1134E3001A800F0D8F8019803990968086601E010
S1134E40684604706846007807B0F0BD00F0FF00C3
S1134E50E9030000F0B50300002210000C00641EFA
S1134E6014D0641E1CD0FE3C24D080256D00641B2D
S1134E702BD08025AD00641B32D08025ED00641B4F
S1134E8039D080252D01641B40D04AE0012425003F
S1134E901E68B7692F40AF4200D12200100040E0E5
S1134EA002241D68AE692640A64201D101263200C3
S1134EB0100036E0802464001D68AE692640A642D6
S1134EC001D10126320010002BE08024A4001D68CB
S1134ED0AE692640A64201D101263200100020E02E
S1134EE08024E4001D68AE692640A64201D1012653
S1134EF03200100015E0802424011D68AE692640AC
S1134F00A64201D10126320010000AE08024640187
S1134F101D68AE692640A64201D101263200100068
S1134F20FFE7C0B2F0BD70B40A0003689D6D524C37
S1134F302C401500EDB22E04F8256D0335402543B1
S1134F409D6570BC70470268520052080B00DBB2CA
S1134F50DB0713430360704710B40268474B1340E8
S1134F600A00D2B292078024E40522401A43026068
S1134F7010BC704710B40268414B13400A00D2B20F
S1134F80D406E022920522401A43026010BC704706
S1134F9010B402683B4B13400A00D2B21406C0227C
S1134FA0920422401A43026010BC704710B4026895
S1134FB0354B13400A00D2B2D20580242404224087
S1134FC01A43026010BC704700B502680B00DBB2E4
S1134FD0012B04D18023DB031343036002E02B4B3A
S1134FE01340036000BD00B502680B00DBB2012B67
S1134FF004D180239B031343036002E0244B13403A
S1135000036000BD10B40268224B13400A00D2B200
S113501012058024640322401A43026010BC7047C6
S113502000B502680B00DBB2012B04D180231B0303
S11350301343036002E0184B1340036000BD00B546
S113504002680B00DBB2012B04D18023DB02134383
S1135050036002E0114B1340036000BD10B402680A
S11350600F4B13400A00D2B21404C0229202224011
S11350701A43026010BC7047FFFFE0FFFFFFFFBF51
S1135080FFFFFFC7FFFFFFFCFFFF7FFFFFFFBFFF27
S1135090FFFFDFFFFFFFEFFFFFFFF7FFFFFFFBFF58
S11350A0FFFFFCFF0268120B12030B009BB21B05EF
S11350B01B0D13430360704710B504000800110072
S11350C00200200000F02AF8200010BD70B4103A4D
S11350D003D378C9103A78C0FBD2530701D318C957
S11350E018C001D508C908C0D20704D30B880380AF
S11350F0891C801C002A01D50B78037070BC704792
S11351008B0701D18307E1D0124205D00B78491CEB
S11351100370401C521EF9D1704700001206130A96
S11351201A43130C1A4300BF094205D0830705D064
S11351300270401C491EF9D1704700001300103959
S113514006D330B41400150010393CC0FCD230BC76
S1135150490700D30CC000D504C0890002D30280E3
S1135160801C002900D502707047000000B50100C2
S113517008000200D2B2802A01DB7F221000C0B2F4
S113518000BD00B501000800C0B2F12805DB08002D
S1135190C0B2FA2801DA012006E00800C0B2802873
S11351A001DA080000E00020C0B200BDFEB582B004
S11351B0070000252C006E463F2030703078694689
S11351C0097AF0220A43024032706846007B70700C
S11351D06846007CFFF7CAFFB0703878002810D00A
S11351E0032004002000C0B2082804DA2000C0B262
S11351F03554641CF6E708226946F868BB6D984785
S113520004E003226946F868BB6D984740B205B0D4
S1135210F0BDFEB506000020050001006A460F231C
S113522013701378F48AF02727431F401770040083
S11352302100C9B2F38A89B2994209D231692300A3
S1135240DBB2C95C2300DBB2D3185970641CEFE7EE
S11352503178002916D005002800C0B20721F38A4E
S1135260C91A884208DA2800C0B2F18A4018101816
S1135270CC2141706D1CEFE708226946F068B36DDC
S1135280984706E0F28A521CD2B26946F068B36DC0
S1135290984740B2FEBD3EB5050068461F21017027
S11352A00178EA8A92B2120AF02313430B40037086
S11352B0E98A417000242100C9B2E4B22100C9B2D4
S11352C0062909DA29692200D2B2895C2200D2B205
S11352D082189170641CF1E708226946E868AB6D96
S11352E09847010049B2002904D1298B891D2983DB
S11352F00121A97640B23EBDFEB506000027390063
S1135300C9B201A82F2202700278B37EF0241C4394
S113531014400470F28A338BD21A6B461A806A46A0
S11353201288082A02DB07226B461A803C00E4B28A
S11353302100C9B26A46128889B291420BD23169FE
S1135340328B2300DBB2D218895C2200D2B28218DD
S11353505170641CECE7317800291BD03900C9B2C4
S11353603D00EDB22A00D2B207216B461B88C91A50
S11353708A4209DA2900C9B26A4612888918411892
S1135380CC224A706D1CEDE7082201A9F068B36DC8
S1135390984707E068460288521CD2B201A9F06817
S11353A0B36D9847010049B200290BD1318B6A468D
S11353B0128889183183B17E491CB176B17E1029D7
S11353C000DBB77640B2FEBDF8B504000D00160050
S11353D000210F000F202B780200134206D0320068
S11353E0D2B2521E2B7803409A4208DA606D00282C
S11353F002D0A248616D88470620C04315E02A7890
S113540010404222A0520800C0B24222A25A80B2E6
S1135410904209D20800C0B228184078E26B0B0011
S1135420DBB2D054491CEEE70020F2BDF8B504000D
S11354300D001700002108006A4610703800C0B241
S1135440082808D0606D002802D08D48616D884717
S11354500620C04339E028780002F02212010240FD
S113546068781618300080B2082808DA606D0028C1
S113547002D08448616D88470620C04325E040205F
S1135480205A320092B2904208D2606D002802D0B5
S11354907D48616D88470220C04316E042202652B1
S11354A00800C0B2062809DA0800C0B228188078BB
S11354B0E26B0B00DBB2D054491CF1E70620442216
S11354C0A05201204622A0540020F2BDF4B50500EC
S11354D00C00002217004620285C21780907090FD8
S11354E0884202D00320C04340E04220285A44218D
S11354F0695A461A300080B2082801DB07200600EA
S113550068460078401E310089B2884208DA686D26
S1135510002802D05D48696D88470620C04325E015
S113552011000800C0B2330080B29BB298420CD282
S1135530E86B0B00DBB24427EF5BDB190F00FFB213
S1135540E7197F78C754491CEBE74420285A80198F
S11355504423E8524620285C401C4623E854462055
S1135560285C102801DB46202A540020F2BD70B5C7
S113557004000D0016003000C0B2032808DA606D84
S1135580002802D04248616D88470620C04300E0ED
S1135590002070BD70B504000E0015002B009BB2F6
S11355A03200E168200000F001F870BDFEB504008F
S11355B000263700002C02D10020C0435CE0A08A02
S11355C069460989884208D2606D002802D03148B2
S11355D0616D88470220C0434EE03420205C0128DE
S11355E008D1606D002802D0C948616D8847012048
S11355F0C04341E068460089E082300020833500E2
S11356002800C0B26946098980B2884209D201984B
S11356102900C9B2405C21692A00D2B288546D1CA9
S1135620EEE7E08A082804DA2000FFF7F2FD07001D
S113563020E02000FFF72FFE0700380040B20028CA
S113564018D13000A0833000A0773000E077E06DFF
S113565080472200203203C2083AE06D80470022CE
S1135660643051412200283203C2083A26630120E3
S113567034216054380040B2FEBD00003CBB000041
S113568068BB000000BA000038BA0000F0BB00009C
S113569010BC000070BA0000FFB583B00400684677
S11356A0007E022803DB6846007E092800DB2CE12B
S11356B000252900C9B22800C0B201006A46127E42
S11356C0C9B2914209D205990200D2B2895C01AAF9
S11356D00300DBB2D154401CEFE72E00F6B23000D9
S11356E0C0B208216A46127E891A884208DA01A8E3
S11356F03100C9B26A46127E89184554761CEEE719
S113570001AF3878C0B20009002806D0022865D05D
S113571021D3032800D1B0E0F7E05120205C012818
S113572004D10520C0435021605401E05020255489
S11357306846027E01A92000FFF746FE694608700C
S1135740694600200856002804D10498A06302206A
S113575051216054D9E05120205C012804D1052056
S1135760C0435021605401E0502025546846027E15
S113577001A92000FFF75AFE694608706946002017
S113578008560221C94388420CD10720C043502146
S11357906054512025540023002202212000FFF7E9
S11357A005FDB2E0694600200856002815D104988A
S11357B0A063012051216054607847216054012383
S11357C04720225C00212000FFF7F0FCE06D8047B9
S11357D0002264305141A064E16496E05120205CD1
S11357E0012804D00520C043502160548DE0049862
S11357F0A16B884200D088E06846027E01A920009F
S1135800FFF764FE694608700320C0436A4600211E
S11358105156814204D1502160545120255474E0E2
S1135820694600200856002826D1E06D80470022F2
S113583064305141A064E1644420205A4221615AF9
S1135840884203D302205121605415E06078002877
S113585012D04720205C401E472160544720205C22
S1135860002809D160784721605401234720225C35
S113587000212000FFF79AFC47E03420205C012837
S113588043D16846027E01A92000FFF770FE6946F5
S11358900870694600200856002835D1E06D80471D
S11358A00022643051412200283203C2083A0F20FA
S11358B039780140022906D10720C0432063022021
S11358C03421605420E03978014001290CD1E07F73
S11358D0401CE077E07F022816DB0620C0432063EB
S11358E00220342160540FE0397801420CD17878D9
S11358F0002802D18448A08301E07878A083B87896
S1135900FFF73FFCA077E577FFE707B0F0BD0000A5
S1135910A4BA0000FEB50100089A00200300512437
S11359200C5D022C02D00420C04328E08C6B8D68EF
S1135930AC4201D1012400E00400009D2C704224FB
S11359400C5B6D462D892600B6B2B54202D26D4677
S11359502D892C0005002B0026009BB2B6B2B34261
S113596009D2CB6B2E00B6B29B5D019E2F00BFB255
S1135970F3556D1CEFE714805123C8540020FEBD7D
S113598070B402000B001878107058785070586882
S1135990506098689060D868D06018691061988ADF
S11359A0908200242000D082200010832000907672
S11359B020009083200090772000D07700200021E1
S11359C01500203503C5083D1500283503C5083DDD
S11359D014632500342695559D69D5639D8B402617
S11359E095532500422695532500442695532500BA
S11359F0462695552500472695559064D164200088
S1135A005021505451201454186A5065586A9065B6
S1135A10986AD06570BC704770B504003420205C6F
S1135A2001285AD1384DA08BA84202D0A08B00285F
S1135A3041D0A07F002810D0A07F00283BD0E06D8B
S1135A40804702000B002000203003C8801A9941CF
S1135A50002930DC01DB00282DD22000FFF74CFCAC
S1135A600600300040B2002822D1A08BA84202D008
S1135A70A08B4019A083E06D80470022643051411F
S1135A802200283203C2083AE06D804702000B006E
S1135A90A07F0021801859412200203203C2083A15
S1135AA0208BE18A884206D300203421605402E02E
S1135AB0022034216054E06D8047220028320CCA51
S1135AC0121A8B41002B08DC01DB002A05D20120CD
S1135AD0C04320630220342160545120205C0128FB
S1135AE011D1E06D8047A26CE36C121A8B41002B3C
S1135AF009DC01DB002A06D20220C0435021605495
S1135B0000205121605470BDFFFF000008B4024B17
S1135B109C4608BC6047C046D1050020F0B5020091
S1135B2052B2002A17D41822AA4B040064B2A40863
S1135B30A4001C59FF25C6001640B540AC438D0196
S1135B40EDB2C600324095402543020052B292089D
S1135B5092009D501BE00F22B74B182405006DB234
S1135B601540083DAD08AE0005006DB22A40083A64
S1135B70920892009A58FF25C7002740BD40AA43C7
S1135B808D01EDB2C7003C40A54015439D51F0BDC9
S1135B9000B5BFF34F8FA948A9490860BFF34F8FE1
S1135BA000BFFDE710B50400601E8021490488424F
S1135BB001D301200EE0601EA249086003210020E9
S1135BC0C043FFF7ABFF0020C54908600720C54963
S1135BD00860002010BD00220260416001230372AE
S1135BE04272704700B5017A00290FD0417A00292A
S1135BF00CD101684268914208D20168491C0160D5
S1135C0001684268914201D10121417200BD70B521
S1135C1004000E001500B448215A9520C000201835
S1135C20FFF7D9FF7820205C012806D02A0092B221
S1135C30310020001830FFF7ADFC70BDFEB5050043
S1135C400E001400082100226F463800FFF766FAA0
S1135C502000C0B2782806D0A348295A9520C00055
S1135C602818FFF7B8FF7920285C002814D02000FA
S1135C70C0B211280FD02000C0B212280BD02000CF
S1135C80C0B2312807D02000C0B27E2803D0200043
S1135C90C0B27F2800D10AE068467F2101704670B7
S1135CA084700322694628001830FFF773FCF7BD9F
S1135CB010B504009020C000201803C80022401C26
S1135CC051419022D200A21803C2083A9220C00087
S1135CD02018FFF787FFB7482018FFF783FF9520A8
S1135CE0C0002018FFF77EFF10BDB34803C87047FB
S1135CF080B5B2480168491C0160AF4A03CA083A3A
S1135D000023401C594103C2083AAD48FFF7D0FFB5
S1135D1001BDF8B596B0002000216A461170A94C67
S1135D2068460078CC21615C884250D2684600788D
S1135D3069460873A44D03A92868FDF7B7FE002837
S1135D403FD0D02020586946097814225143401886
S1135D50407A012831D103A92868FDF761FE03A91F
S1135D602868FDF7FAFD03AC4820205C029003A8E4
S1135D7008300190BD4DA02040002E183078142129
S1135D8048432818071D029A01993800FFF7B8F90B
S1135D9004983178142251436850307814214843D0
S1135DA028184821615C01733078401C30703078C9
S1135DB0102806D30020307003E003A92868FDF7FB
S1135DC02FFE68460078401C69460870A7E717B0A4
S1135DD0F0BD000000E400E080B5FFF79AFF01BDCC
S1135DE080B5FFF796FF01BDF1B582B00024684687
S1135DF004709E48FF2142314518A0214900415CAE
S1135E002A78914215D01426297814225143401837
S1135E100190029F320001993800FFF771F9287848
S1135E20401C28702878102800D32C700120694663
S1135E30087068460078FEBD1CED00E00400FA0519
S1135E400CED00E014E000E0F3B595B01700002479
S1135E502600F6B22000C0B2E4B25A482100CC2297
S1135E60825CC9B291420ED21599D0228258230085
S1135E70DBB214256B43D2185268914201D126003B
S1135E8001E0641CE9E7D03002A902683300DBB208
S1135E9014256B43D25A0A7048228F54006831008B
S1135EA0C9B2142251434018406803903800C0B26C
S1135EB001901698009002A805000835019A0099EF
S1135EC02800FFF71DF9944D02A92868FDF7F6FC98
S1135ED002A92868FDF7E4FC002017B0F0BD00001B
S1135EE018E000E010E000E08C040000FEB500249F
S1135EF00294354F894D28007C3038602E00BC3622
S1135F0006220F21300000F08CFA06220E21300008
S1135F1000F087FA01202B4E0100317021007170CE
S1135F202100B17030217454C821705402AA0B218D
S1135F3028000830FCF79DFE707801280BD1012061
S1135F400190FA20C0000090754B764A0299300007
S1135F501C30FDF7DEFE0020019073480090704B6A
S1135F60724A029930000830FDF7D3FE31003868D8
S1135F70FDF7C4F90B2000F03FFB0C2000F03CFBC4
S1135F80F7BDF0B50400200000252E00954209D28B
S1135F90674E4F5D4740FFB2BF00F659000A70409C
S1135FA06D1CF3E71E00F6B2012E02D10026F64363
S1135FB0301AF0BD9C040000081600208C2000203C
S1135FC010160020E4270020BC280020FEB5002580
S1135FD0280069460870574F0C21380000F01EFB5A
S1135FE0002831D10126544C3000207001213800A2
S1135FF000F014FB012827D10220207008212A0078
S113600001AC2000FFF78AF8082201A94B48FFF7EA
S11360107DFD002818D1494C20684949884213D194
S11360202F00082201A98D208000FFF70DFF280012
S11360300100C9B2042903DA2560241D401CF7E7D6
S113604040490D6069460E706846007800280AD100
S113605028003A4A29000800C0B2042803DA15606F
S1136060121D491CF7E768460078FEBDA0260020F3
S1136070FEB50026019600963700304C00F0B0FAC9
S113608025480068FDF790F82F4800F0BCFA0B2073
S113609000F0B9FA0C2000F0B6FA35002800C0B2BE
S11360A0042803DA2660241D6D1CF7E780204002D3
S11360B00768264806682648066026490F600A686D
S11360C082F30988096881F3088880214902BD4A5E
S11360D0116000688047F7BDBB494870704780B5C0
S11360E0FFF756FD01BD0020C0B2704738B505006A
S11360F00C00220092B22900B348FFF788FD31BD9D
S113610038B505000C002200D2B22900C9B2AE484D
S1136110FFF794FD31BD0000BC280020301F002093
S11361204C1D000080841E00C409000020A107004B
S1136130909900001C200020062E0020F03F002033
S113614055AAAA5500160020FFFF00000400010014
S1136150C4280020C028002010B504002000C0B2CC
S1136160012802D100F02EFA01E000F039FA10BD46
S1136170F8B590B000F034FA944E300000F00EFB05
S1136180AC204000301800F035FC914C200000F0A9
S113619076FC210030005C3000F080FC8D4B012245
S11361A0002130005C3000F010FDA220400005907A
S11361B000200490884C049A05992000FEF7AEFF55
S11361C0D820039000200290844F3C00029A039947
S11361D02000FEF7A3FF06AC0120207002206070AF
S11361E00120A0807E4D06AA07212800FCF75EFD51
S11361F0012020700120A08006AA13212800FCF7AA
S113620055FD06AA14212800FCF750FD06AA152105
S11362102800FCF74BFD012020700720607006AABF
S113622025212800FCF742FDA02040003018006E14
S1136230009002216846FEF79DFE00F07BFD00F011
S1136240C3FE3800FCF736FF0420CC21785465489F
S1136250D0217850FFF74AFE63495B4800F05CFFA9
S1136260624930005C3001F016FA614C22000921C9
S11362702800FCF7FEFC2068FA218900FCF77DFD6C
S1136280FFF790FC5B4800F0B7F900F09BF9BC36CF
S113629001220621300000F0C4F80022062130005B
S11362A000F060F901220721300000F0BAF8002262
S11362B00721300000F056F901220821300000F0D7
S11362C0B0F800220821300000F04CF90122092125
S11362D0300000F0A6F800220921300000F042F955
S11362E001220A21300000F09CF800220A2130002B
S11362F000F038F901F04EFC3F49002001F0A6FE01
S11363003E480168002948D0002404603C4D2868B8
S1136310401C286028680A21FCF72FFD002901D1C0
S113632000F020FE2868FA218900FCF726FD0029E8
S113633011D1032000F024FE070032490120087126
S1136340380080B2000A48713800887108228D2014
S11363508000FFF779FD28682B49884208D32C6018
S11363602A480168002902D10121016000E004608B
S1136370300000F006F98009C006C00E01900198B3
S11363800E2802D1012001F0C7F9012001F0A4FA7E
S11363900D4801F098FF01F08FFA0BA8FFF724FDD8
S11363A00128ADD10B981A49884203D00B9819499A
S11363B08842A5D10BA8037B021D0B991648FFF751
S11363C06BF99DE708ED00E010160020301F002057
S11363D0D02800208C080020A0260020E4270020DC
S11363E0381F002024B9000050080020D8BA00004B
S11363F098200020FFFF0000C8BC00008C20002073
S113640090200020C8280020881300009420002039
S113641032070000DF0700002816002001604260F8
S11364207047F5B58BB00CA8007800286ED10CA885
S113643000786A46107106910B980068069A9200DB
S11364408258474B13406A4612791202E024E40052
S113645014401C430A940A9A069B9B00C2500025D0
S11364606A46D57005910B9A1268059B9B00D35818
S11364700224A3436C46E4786400022634401C439F
S11364800994099B059CA40013516B469D700491CB
S11364900B9B1B68049CA4001E590124A6430124E1
S11364A06F46BF78274037430897089E049FBF0074
S11364B0DE516E46757003910B9D2D68039EB600E8
S11364C0AF598026B743BC466E467678F6018027DE
S11364D03E4067463E430796079E039FBF00EE512A
S11364E06E46347002910B9C2468029EB600A75934
S11364F00426B743BC466E463678B60004273E40B1
S113650067463E43029FBF00E65127E00020019109
S11365100B9A1268019B9B00D3580424A3430400E4
S1136520E4B2A40004252C401C430294029B019C69
S1136530A40013510CAB1B786C4623700B000B9C0E
S113654024689D006659064D35406E4636783702FC
S1136550E026F6003E402E439D0066510DB0F0BD8E
S1136560FFF8FFFF30B443685B6901248C40A34308
S11365701400E4B28C401C43230045686B6130BCBA
S113658070470100486800697047000000B50100C9
S113659049B2002905D40121C206D20E9140134A02
S11365A0116000BD00B5010049B2002909D40121E0
S11365B0C206D20E91400E4A1160BFF34F8FBFF353
S11365C06F8F00BD00B50B480168012906DB016827
S11365D0491E01600068012800DA62B600BD0000AF
S11365E072B604480168491C0160704700E100E08C
S11365F080E100E02C1F002010B50400200040B210
S1136600FFF7C4FF10BD10B50400200040B2FFF72F
S1136610C9FF10BD016042608360704730B502005D
S1136620002318000C00E4B20D2C01DBC0B2B4E06E
S11366300C00E4B2002C14D0022C29D01CD3042C5E
S11366403ED031D3062C53D046D3082C68D05BD32C
S11366500A2C7DD070D30C2C00D191E000D283E0C1
S11366609AE0156801242D682540EDB2012D01D171
S1136670200000E018008FE0156801242D686D08E3
S11366802540EDB2012D01D1200000E0180083E087
S1136690156801242D68AD082540EDB2012D01D106
S11366A0200000E0180077E0156801242D68ED084B
S11366B02540EDB2012D01D1200000E018006BE06F
S11366C0156801242D682D092540EDB2012D01D155
S11366D0200000E018005FE0156801242D686D09B2
S11366E02540EDB2012D01D1200000E0180053E057
S11366F0156801242D68ED092540EDB2012D01D165
S1136700200000E0180047E0156801242D682D0AD8
S11367102540EDB2012D01D1200000E018003BE03E
S1136720156801242D686D0A2540EDB2012D01D1B3
S1136730200000E018002FE0156801242D68AD0A40
S11367402540EDB2012D01D1200000E0180023E026
S1136750156801242D68ED0A2540EDB2012D01D103
S1136760200000E0180017E0156801242D682D0BA7
S11367702540EDB2012D01D1200000E018000BE00E
S1136780156801242D686D0B2540EDB2012D01D152
S1136790200000E01800FFE7C0B230BDF0B58BB0B8
S11367A00400694D2A006949200001F00BFE684885
S11367B00590069000200790089009900A90654F74
S11367C005A80390029764480190644800902B0048
S11367D0634A644920000830FCF724FA6249200027
S11367E0383001F0F2FD614920003C3001F0EDFD4C
S11367F05F492000403001F0EBFD5E4A5E49200015
S1136800443001F0E7FD5D492000503001F0E6FD21
S11368105B492000543001F0E3FD5A492000583010
S113682001F0E0FD2A00584920005C3000F00CF92A
S1136830022069460874554E04A8039002960197F5
S11368400095474B444A524920007C30FCF722FC17
S113685050492000983001F0C7FD4F4920009C307A
S113686001F0D2FD4D492000A03001F0CFFD4C498C
S11368702000A43001F0CCFD4A492000A83001F0EA
S1136880C7FD49492000AC3001F0C4FD4749200050
S1136890B03001F0C1FD464A46492000B430FFF74C
S11368A0BDFD454A45492000BC30FFF7B7FD444AC9
S11368B044492000C430FFF7B1FD0095274B3A004E
S11368C041492000CC3001F0A9FD32003F492000AD
S11368D0DC3001F049FE32003D492000E43001F093
S11368E043FE1F4B1C4A1F492000EC30FFF792FE69
S11368F038492000F83001F06DFE3749A0204000EF
S11369002018FEF74DF93549A22040002018FEF763
S113691047F932003249A4204000201801F064FEF7
S11369203049A8204000201801F062FE2E49AA2018
S11369304000201801F05CFE2C49AC2040002018D7
S113694000F056F80BB0F0BD00E006400000074030
S113695000127A0000E8064000F8064000E4064011
S113696000F0064000F007400030004000400040C6
S113697000C0004000100240008000400090014030
S113698000800140005000400000024000F005403B
S11369900080034000B007400070074000500740EB
S11369A0000003400010034000D0004000100740E6
S11369B000500340000006404050034000100640D1
S11369C0805003400020064000D00740008005406E
S11369D0009005400080074000C0024000D0024003
S11369E000E0054000A0064000B0064000A00740BB
S11369F00160704710B502680121126852090A400B
S1136A001300DBB2012B19D10D4B046863600368DA
S1136A101B688024A343046823600A4B0468A360B2
S1136A2003681B68DB0A0B40DBB2002BF8D1036858
S1136A301B685B0A0B40DBB2002BF8D010BD0000D2
S1136A4020C528D9FFFF0000F8B504000F00150089
S1136A50276065600026A660E0208002E060802058
S1136A6040052061802000026061200000F053F99D
S1136A702076E661207E002800D06661F1BD002109
S1136A800160E022920242608022520582608022EC
S1136A901202C2600A0002744161704770B50500B9
S1136AA00C000026AE60E0208002E86080204005F3
S1136AB02861802000026861280000F02CF9287603
S1136AC06069E861287E002800D06E6170BDF1B471
S1136AD089B0012069460871099909680791002164
S1136AE006916A461279520002231A400692069AC7
S1136AF0079B1A606A46D070099A126805916B4622
S1136B00DB781B01102423400593059B13606B461F
S1136B109870099B1B6804916C46A4786401202535
S1136B202C400494049C1C606C466070099C24688E
S1136B3003916D466D78AD01402635400395039D64
S1136B4025606D462870099D2D6802916E46367841
S1136B50F60008273E400296029E2E60099E366883
S1136B6008910100C9B289000427394031600AB094
S1136B70F0BC7047F0B50100002528000122130085
S1136B800C681E00F6B2F60180273E4026600B68B2
S1136B901B68DB091340DBB2002BF8D00B681B68C1
S1136BA05B091340DBB2002B0CD10B681B681B097B
S1136BB01340DBB2002B05D10B681B681340DBB21A
S1136BC0002B00D01000C0B2F0BDFFB58BB0002484
S1136BD0270025000D98802801D3012007000E9876
S1136BE0002801D1012007003800C0B2002800D0DD
S1136BF08DE00B98006801260068C1093000084048
S1136C00C0B2002802D10220070080E00B98FFF7F1
S1136C105EFF0920694608712000694648700B9898
S1136C20006809900494FF20089009996A465278F4
S1136C308918097F089A91436A461379089A1A4079
S1136C400A430492049A09996B465B78C9180A7737
S1136C500D996A46D17069460E700B9909680791BF
S1136C600394069007996A4612788918097F069A50
S1136C7091436A46D278069B13400B4303930399CE
S1136C80079A6B461B78D21811770CA909786A46C3
S1136C90917002210B9A1268029405900B00DBB2EA
S1136CA0D3181E7F059B9E43B4466B469E78059B76
S1136CB03340664633430293029B0E00F6B29619A4
S1136CC033772500082D1ED20E99495D6A4611704E
S1136CD02900091D0B9A1268019402900B00DBB283
S1136CE0D3181E7F029B9E43B4466B461E78029BBC
S1136CF03340664633430193019B0E00F6B2961966
S1136D0033776D1CDEE70B98FFF734FF070038007C
S1136D10C0B20FB0F0BD10B5010000231A000C681A
S1136D2001202468640C0440E4B2012C00D0180053
S1136D30C0B210BD18B589B000F042F86846FDF73E
S1136D40BBFE012069460872804A01920022CA7281
S1136D5048727F4C6A46252120000830FBF789FFE2
S1136D600028F6D0A0204000241869462000FDF732
S1136D70D5FE00212000FEF7D6F800200AB010BD91
S1136D807CB506000D00734B1E705D70724C009450
S1136D90022201217148FDF797FF207800026178F3
S1136DA0084380B276BD10B56C4C02212000FDF77B
S1136DB019FF012803D102212000FEF74BF810BD72
S1136DC0F0B595B0664C07220C212000FFF729FB93
S1136DD001256846C5710C200E9021680D910D990E
S1136DE00E9A92008958402291436A46D2799201C0
S1136DF040231A400A43149214990D9A0E9B9B0047
S1136E00D15069468D710C9020680B900B980C99A9
S1136E10890040582027FF43384020266946897955
S1136E20490131400143139113980B990C9A920034
S1136E30885007220B212000FFF7F3FA68464571BA
S1136E400B200A902168099109990A9A920089589D
S1136E50402291436A465279920140231A400A43E0
S1136E601292129B09990A9A92008B5069460D71ED
S1136E70089020680790079808998900405838407E
S1136E8069460979490131400143119111980799E3
S1136E90089A9200885007220A212000FFF7C1FABD
S1136EA06846C5700A200690216805910599069ADE
S1136EB092008958402291436A46D2789201402335
S1136EC01A400A431092109B0599069A92008B501F
S1136ED069468D7004902068039003980499890092
S1136EE040583840694689784901314001430F913F
S1136EF00F980399049A92008850072209212000D0
S1136F00FFF78FFA68464570092002902168029ABB
S1136F1092008B58402293439C466A4652789201D1
S1136F2040231A4063461A43029B9B00CA506B4697
S1136F301D70236884001C5927406C462478640122
S1136F4026403E4384001E5115B0F0BD40420F0060
S1136F50301F0020A02D0020AC2D00207020002028
S1136F60E41F00201CB5032000F00AF804000022EE
S1136F702100C9B2032000F00BF80090009816BD60
S1136F8010B5040000216006400EFFF7F9FE10BDA5
S1136F90F8B505000C0017002100C9B28020284371
S1136FA0C0B2FFF7EDFE0600002F00D03E80684619
S1136FB005702800C0B2FFF7E3FF604069464870DF
S1136FC0684684700098F2BDF0B599B01527380072
S1136FD0002529006A4651710100C9B209094140DE
S1136FE00800C0B2800848400100C9B249084140C5
S1136FF068460171684600790100C907C90F012973
S113700001DB952007002C000495200080B2C00805
S113701069464873200040016946087328006946A0
S1137020C8722800694688720498C0086946487284
S1137030049840016946087228006946C87128000E
S11370406946887105A833495022FEF73FF805AE1A
S113705077706846407B292170546846007B2B2159
S113706070546846C07A2D2170546846807A2F2166
S113707070546846407A312170546846007A33214E
S113708070546846C0793521705468468079372138
S11370907054684640794B217054FFF74BFE00282A
S11370A009D0280069460870FF2069464870684680
S11370B0857000982BE02C002000C0B24000305CAA
S11370C0002806D12000C0B24000301840780028C3
S11370D014D000222000C0B24000301841782000B3
S11370E0C0B24000305CFFF753FF00906846407820
S11370F0002801D000980AE0641CDDE728006946F6
S1137100087028006946487068468570009819B070
S1137110F0BD000074B9000038B505000C00210072
S1137120280001F095F80548A8600548E8600C209F
S11371306860044828610620A88231BD0CB80000AC
S1137140BCBB0000FC080020F3B581B01400C025CE
S11371502600F6B2281D0090029F320000993800E4
S1137160FDF7CEFFF7BD43780B707047F3B581B0E0
S11371701400C0252600F6B2280028300090029F93
S1137180320000993800FDF7BBFFF7BDF5B583B0B9
S11371900C00C0250C200290280018300190260015
S11371A0029A01993000FDF7ABFF082628000C3045
S11371B0009027000C37320000993800FDF7A0FF3B
S11371C02020E07205B0F0BDF3B581B01400C025F5
S11371D02600F6B20095029F320000993800FDF7B0
S11371E08FFFF7BD30B500231C001500E4B2EDB2EB
S11371F0AC4205D220241D00EDB24C555B1CF3E7D4
S113720030BD00008020C000704770B5C024240148
S11372100025894E2A0021003000FDF77FFF70BD54
S113722010B5002485484068006A8047C0B210BD8C
S1137230704710B5814C607A002820D18A20C000A4
S1137240205C012803D07E48205C01280DD1002059
S11372508B21C9006050012079496054022060727A
S1137260022061680969884709E0042000F040FAB7
S113727001208721C900605402207249605410BD66
S1137280F8B584B06D4C607A002802D0607A012889
S11372906AD16069002867D0A0696169884263D2B5
S11372A000252E00E7686848205C012831D00020C2
S11372B06168096888470121E0688022D20080184B
S11372C06268926A904706003000C0B200280AD172
S11372D0782131206268926990470121E0686268F0
S11372E0926A904706003000C0B200280DD1782180
S11372F031206268926990476169891E802000018B
S113730038186268926A904706000120616809682B
S113731088473000C0B2002812D102A84B490CC9DA
S11373200CC0083908380220607265612561A561C6
S113733002A80571052102A862685269904713E00A
S11373406846C0490CC90CC0083908386561256114
S1137350A561032000F0CCF90120694608710521DC
S1137360684662685269904705B0F0BDFEB5384E74
S1137370307801285FD13148407A002803D02F4863
S1137380407A012857D12D4CC148205C012852D1A4
S1137390606A216A88424ED2002528006946087036
S11373A02948205C012813D00020616809688847B7
S11373B08022D20021002D31E069636AC01863681D
S11373C0DB6A984769460870012061680968884744
S11373D068460078002821D108212A0001AF38002E
S11373E0FDF79CFE606A8021C90040186062606AF3
S11373F0216A884204D3280030700220607201E0C0
S11374000120607201A8762101702C21615C417019
S1137410022101A86268526990470AE0280030708E
S11374202562656228002C216054A562032000F0C7
S11374305FF997482554F7BDF0330020C81A00209F
S1137440540400004404000055040000ECBC000097
S1137450FD1E0020FEB5A54C607A002803D0607A9A
S1137460012800D0EDE0607A002822D1A648201837
S11374700178002900D0E4E0A4490D68A44A9542AB
S11374800DD3DC229202954209D2B1480268086801
S1137490A04941188020400200F0E6F9D1E0012122
S11374A00170022060720020AA496054A44960540B
S11374B0C7E0607A012800D0C3E0A14825182878E5
S11374C0022800D090E0904826183078012854D142
S11374D001238820C00022589F4821580020C0431F
S11374E067687F68B8479D4908609C48006889219F
S11374F0C9006158884237D10020C04300908349B5
S11375000F6883498F4208D3E02189028F4204D255
S1137510391F019101990968009191490968A54AA7
S1137520914207D10099A44A914203D1884909683C
S1137530814208D101203070002086496054022124
S1137540617228705CE001200100824AA154317804
S1137550002903D1052000F0CBF851E0307002205F
S11375606072002028704BE00120307002206072AD
S1137570002078496054287042E00020C043009005
S113758062490F6862498F4208D3E02189028F4221
S113759004D2391F01910199096800917049096861
S11375A0844A914207D10099834A914203D16849A0
S11375B00968814208D10120307000206549605477
S11375C00221617228701BE0002062496054317806
S11375D0002903D1052000F08BF811E0012131705E
S11375E00221617228700BE02878012808D1FFF786
S11375F01FFE012057496054022060720020287049
S11376008720C00020180178002918D168469549C0
S11376100CC90CC0083908384E48205C012803D135
S113762000206946087102E00120694608710521BD
S113763068466268526990470220607201E0002146
S11376400170F7BDF4BC000010B5284C607A002826
S113765002D0607A01281AD19648205C012805D10D
S1137660FFF7D3FD6068C069804710E08B20C0003D
S113767020581E2809D32448205C002805D1FFF790
S1137680C4FD6068C068804701E00120607210BDDD
S1137690360400007047F2B582B006008C20C000AA
S11376A0019000250095114C2700009A019938009B
S11376B0FDF734FD0298606026608620C0002550E6
S11376C030006168496A88470F48271860688068F5
S11376D0804738703878012806D18B20C0002550A7
S11376E00220616809698847F7BD0000C81A0020B4
S11376F00021894A0B00537210728B23DB00D15096
S1137700704786480078704754040000F87F0300EF
S1137710010001000000FFFF10B57F49804A8A186C
S11377201378002B08D18A23DB00C85400238B2450
S1137730E4000B510123137002224A7210BD0000B1
S113774044040000744A774BD054774BD1547047AB
S1137750FC7F03004C0400003C040000281F0020B0
S1137760C000010038B505000C006B480461C56019
S113777000216E4A81546E4A8154802149028D420F
S11377800CD1A02189028C4208D10221694A81547A
S11377900169694A8918890A416107E067498D428C
S11377A004D10121634A8154032141610120FFF77F
S11377B09FFF31BDDDCCBBAAAABBCCDD70B50500F3
S11377C00C00012054495A4A885400221300574E91
S11377D08B55CD610C624A628A622C23CA54802282
S11377E0520295420AD1C022D201944206D3544A8D
S11377F0944203D202204F4A885404E04F4A9542EF
S113780001D14C4A88540220FFF772FF70BDF7B5CE
S113781000221300100011006B469B88994209D284
S11378203D4B9C6A64181B192D24009D6D5C1D55ED
S1137830491CF1E7384B434C9D6A6E46B688AD1936
S113784025606D462D7A2C269D559D6A8026F6006E
S1137850B54205D301252E00344FDE5528002260A1
S1137860C0B2FEBDFCBC000070B52B4B01245C72A1
S113787004251D728925ED005A518825ED005951C2
S1137880314D58510025314E9D5580256D02A84239
S11378900AD1C025ED01A94206D32D4DA94203D238
S11378A002242C4D5C5504E0244DA84201D1294DFD
S11378B05C5570BD5204000080B51748017A062952
S11378C009DA2549027A92008A58002A03D0007AFC
S11378D080000858804701BD10B504000E48017AA5
S11378E0002902D0017A052907D18B21C90041184A
S11378F00A682300DBB2D2180A600A4941180A78E0
S1137900012A07D100220A700121144A815405205A
S1137910FFF7EEFE10BD0000C81A0020141F00205F
S11379205404000051040000530400003604000015
S11379303504000055040000FF030000F03300206C
S113794001800200F01A00203C0400004C040000F6
S113795001700200440400003808002052040000B2
S113796010B55B4C0320206160615A48A0615A49FC
S1137970E1618021C90021620021A1626162E162AA
S11379802066564860661020A0662167E16661673C
S113799053A1E01D00F052FE5249200000F04EFEBB
S11379A02020A07110BDF1B586B00C001500002098
S11379B001900698C768069800690090009887426D
S11379C003D20098C01B401E05E006988068C01BC7
S11379D000994018401E06998968C91B884202D341
S11379E006988068C01BA84201D2060000E02E0061
S11379F006984068C0190390059604940398029071
S1137A00059A04990298FDF77BFB02980198801966
S1137A100190A419AD1BBF1906988068874201D153
S1137A20002007000698C760002DC4D1019807B054
S1137A30F0BDF8B588B004000D001600E0680390AE
S1137A40A0680399401A0290029886420FD2606897
S1137A5003994018009005960495009F059A04998F
S1137A603800FDF74DFB03988019E06020E0029890
S1137A70019060680399401800900198079006955A
S1137A80009F079A06993800FDF73AFB0298301ACE
S1137A90019060680090019805900298281804905D
S1137AA0009F059A04993800FDF72AFB0198E060CD
S1137AB009B0F0BD00B501000A69CB68934204D354
S1137AC08868401EC01A801801E0D01A401E00BD0C
S1137AD0E8280020E0BC000090290020902D002020
S1137AE05254540004BD0000F1B582B00F001500DB
S1137AF00197274802991822514340180600183666
S1137B007069002803D0022821D010D326E0300069
S1137B10FFF7D0FF00900098A84201D2002405E0AE
S1137B202C002A0001993000FFF783FF17E0300092
S1137B30FFF7C0FF00900098A84201D2009C00E02B
S1137B402C00220001993000FFF773FF07E02A00A0
S1137B5001993000FFF727FF040000E00024200013
S1137B60FEBDF1B50F001600094D2878002801D19B
S1137B70FFF7F6FEEFF31084012080F31088320043
S1137B8039000098FFF7B0FF84F31088F2BD0000BD
S1137B90E828002080B5FFF7E3FE01BD70B50400BE
S1137BA00E00A56861682800401C814207D3206844
S1137BB046552800401CA060E068401CE060A068B6
S1137BC0616888420DD1A26821682069FFF7C9FF66
S1137BD0A168884203D00020C043E06001E0002097
S1137BE0A06070BDF7B584B01F000C9D059802908D
S1137BF00124012602980699884206D30298069920
S1137C00FBF7BBF80290761CF4E7BE4200D23E00BC
S1137C100D98C0071BD4002D19D00D98800705D5E9
S1137C20002F03D130206946087002E02020694605
S1137C300870002D0BD0AE4209D26D1E6846017843
S1137C400498FFF7ABFF0498C0680028F1D50498A6
S1137C50C06800283CD4022F01D37F1E08E0059899
S1137C602100FBF78AF8019001980699884202D313
S1137C7006984443EFE705982100FBF77EF801904E
S1137C80059801996143401A059012480199415C95
S1137C900498FFF783FF0498C068002806D42000E6
S1137CA00699FBF76AF80400002CE4D10D98C0078C
S1137CB00ED5002D0CD0002D0AD0AE4208D26D1E78
S1137CC020210498FFF76AFF0498C0680028F2D5C1
S1137CD007B0F0BDB8BC0000FEB582B007000A9C36
S1137CE00298002802D50298454200E0029D012630
S1137CF00398854206DB28000399FBF73BF805004F
S1137D00761CF5E70498864201D204980600002CFC
S1137D1006D00298002802D40B98400700D5641EB0
S1137D200B98800702D50498002810D00B98C00740
S1137D300DD4002C0BD0002C09D0A64207D2641E0F
S1137D4020213800FFF72AFFF8680028F3D5F868E7
S1137D50002836D40298002807D50298414202919F
S1137D602D213800FFF71AFF06E00B98400703D5D2
S1137D702B213800FFF712FFF868002821D40B9854
S1137D808007800F022810D1049800280DD1002C00
S1137D900BD0002C09D0A64207D2641E3021380033
S1137DA0FFF7FCFEF8680028F3D5F868002808D42B
S1137DB00B9801900094049B039A02993800FFF7F2
S1137DC011FF05B0F0BDF5B59BB00C000AA80590F5
S1137DD040200690002007901B98099000200890EE
S1137DE020780700641C3800C0B2002800D11BE1D1
S1137DF03800C0B2252800D00DE100200500012183
S1137E000291227817003A00D2B2232A13D02B2AE7
S1137E100CD02D2A02D0302A03D011E00D43641C6B
S1137E200FE02A0002251543641C0AE02A000425F9
S1137E301543641C05E02A0008251543641C00E072
S1137E400290029A002ADCD1039021780F003900B5
S1137E50C9B2302903DB3900C9B23A2906DB0490E0
S1137E6020780100C9B22E2920D109E0641C0399AD
S1137E700A2251433A00D2B2891830390391E4E717
S1137E80641C217808000100C9B2302903DB010019
S1137E90C9B23A2900DB09E0641C04990A2251435F
S1137EA00200D2B2891830390491EAE72778380001
S1137EB0C0B26C2803D03800C0B2682803D1641C57
S1137EC020780700F3E73800C0B2252800D19BE0F2
S1137ED058284ED063280AD064281CD070287BD040
S1137EE073285DD075282DD0782842D091E01C9855
S1137EF000681C9908601C98006800681C9909684F
S1137F00091D1C9A11600290029E3100C9B205A895
S1137F10FFF744FE7DE01C9800681C9908601C98DB
S1137F20006800681C990968091D1C9A1160029078
S1137F30019503980090049B0A22029905A8FFF773
S1137F40CBFE66E01C9800681C9908601C980068C9
S1137F5000681C990968091D1C9A1160029001951A
S1137F6003980090049B0A22029905A8FFF73AFEA1
S1137F704FE01C9800681C9908601C980068006811
S1137F801C990968091D1C9A1160029001950398B7
S1137F900090049B1022029905A8FFF723FE38E005
S1137FA01C9800681C9908601C98006806681C9856
S1137FB00068001D1C99086030780700761C3800A2
S1137FC0C0B2002807D03900C9B205A8FFF7E6FD02
S1137FD008980028F0D51CE01C9800681C990860DB
S1137FE01C98006800681C990968091D1C9A116096
S1137FF0029000200190082000900823102202998A
S113800005A8FFF7EFFD04E0252105A8FFF7C6FD4D
S1138010FFE7641C04E03900C9B205A8FFF7BEFD00
S11380200898002800D4DBE6089801280BDB0798A1
S1138030002804D0079A0AA91B98FFF792FD089814
S113804007994018089008981DB0F0BD0CB438B5D5
S113805005000C0004A800906A4621002800FFF7E0
S1138060B2FE01B0029930BC03B0084700210160A0
S113807041600A000272417270470022026041604E
S11380800123037242727047407A7047FEB50500BF
S11380900E001400082100226F463800FDF73EF858
S11380A02000C0B2782806D0C248295A9520C000C2
S11380B02818FFF7E2FF7920285C002814D020005C
S11380C0C0B211280FD02000C0B212280BD020005B
S11380D0C0B2312807D02000C0B27E2803D02000CF
S11380E0C0B27F2800D10AE068467F210170467043
S11380F084700322694628001830FDF74BFAF7BD57
S113810010B5020000231800180080B25468A04281
S11381100CD290681C00A4B22401005D0C00E4B2EF
S1138120A04201D1012002E05B1CEDE7002010BD5C
S113813070B503000024250020002500ADB25E6860
S1138140B5420FD29D682600B6B23601AD5D0E0071
S1138150F6B2B54204D1250015700125280001E0CE
S1138160641CEAE7C0B270BD7CB504000E000025B3
S1138170FF20694608706A463100C9B22000FFF743
S1138180D7FF012861D16078012804D05DD303288A
S11381901FD03CD359E0206D216A88420AD1A068DF
S11381A06946097809014018C078012810D10120D6
S11381B005000DE0206DE169884209D1A068694697
S11381C00978090140180079012801D1012005002E
S11381D03BE0206D216A88420AD1A068694609788B
S11381E0090140184079012810D1012005000DE053
S11381F0206DE169884209D1A068694609780901BE
S113820040188079012801D1012005001DE0206D6E
S1138210216A88420AD1A068694609780901401890
S1138220C079012810D1012005000DE0206DE1691D
S1138230884209D1A0686946097809014018007A82
S1138240012801D101200500FFE72800C0B276BD56
S113825070B505000C00210028001830FDF790FBD4
S11382600120687000263000A8703000782168541E
S1138270002000219022D200AA1803C2083AA08D3F
S11382809121C9006852E08D4B496852208E4949BA
S113829068529220C0002818FFF7E8FE47482818C3
S11382A0FFF7E4FE9520C0002818FFF7DFFE310039
S11382B030004349884205D231002A187B23D15427
S11382C0401CF6E770BDFEB5040000263000694688
S11382D0C880300069460871370035002000183026
S11382E0FDF79AFB01A8801C0090354B22007B32DD
S11382F02100793120001830FDF70CFB6946087124
S1138300694604200856002843D17B20205C0700DE
S11383103900C9B22000FFF7F3FE002833D039003A
S1138320C9B22000FFF720FF012832D13500606870
S113833085422ED2A0682901405C3900C9B2884226
S11383401FD1A068290140188078002806D07C201D
S1138350205CC0B2C0097821605402E0300078216A
S1138360605428007A2160546846C28821007B3119
S113837020000400A36828011818C3682000984747
S113838007E06D1CD3E711223900C9B22000FFF7C2
S11383907DFE9520C0002018FFF776FE012807D146
S11383A001206070A6709520C0002018FFF75EFEC3
S11383B0F7BD00008C0400008A0400009C04000047
S11383C002040000016042607047016070470000D1
S11383D0016070474160826070470000016070472F
S11383E00160704701607047F0B4016000220368C7
S11383F0DC6E65086D00DD6605682E6C3700FF07CE
S1138400FF0F2E6CF0BC704701607047016070472D
S113841001607047016070470160704710B4019CAF
S1138420016042608360C46010BC704710B402698C
S1138430584B13400A00D2B21405F0221204224011
S11384401A43026110BC704710B40269524B1340C6
S11384500A00D2B21404F022120322401A43026129
S113846010BC704710B402694C4B13400A00D2B2DE
S11384701403F022120222401A43026110BC704716
S113848010B40269464B13400A00D2B21402F0221F
S1138490120122401A43026110BC704710B40269F1
S11384A0F0239A430B00DBB21C01F0232340134357
S11384B0036110BC704702690F239A430B00DBB2BF
S11384C01B071B0F13430361704710B44269314B00
S11384D013400A00D2B21405F022120422401A43B7
S11384E0426110BC704710B442692B4B13400A0020
S11384F0D2B21404F022120322401A43426110BC87
S1138500704710B44269254B13400A00D2B21403D9
S1138510F022120222401A43426110BC704710B488
S113852042691F4B13400A00D2B21402F022120116
S113853022401A43426110BC704710B44269F023D0
S11385409A430B00DBB21C01F02323401343436125
S113855010BC704742690F239A430B00DBB21B0720
S11385601B0F134343617047F8B505000F00160055
S11385702F606E600024200080B20C2809D21348BA
S1138580210089B2425C0C21280000F00BF8641C25
S1138590F1E7F1BDFFFF0FFFFFFFF0FFFF0FFFFF4C
S11385A0FFF0FFFF70B505000C0016003000C0B2EC
S11385B00C2808DA2100C9B26868054A3300DBB226
S11385C09B00D258904770BD00000000D4BC00004E
S11385D00CBB000001600022027142712823C254C6
S11385E03823C254704700000160426070470000A5
S11385F0F0B401600268D36A802424021C43D4626C
S113860000BF00BF00BF00BF0A4C1C40D462046816
S1138610E56A8026F6012E43E66200BF00BF00BF74
S113862000BF054E2E40E662002607683E60F0BC9F
S113863070470000FF7FFFFFFFBFFFFF31B48B07D0
S113864007D00B780370002B20D0401C491C8B07EB
S1138650F7D1164CE501830722D104C9131B9343B8
S11386602B4205D104C004C9131B93432B42F9D0F8
S1138670FF231A42027009D0120A1A42427005D02E
S1138680120A1A42827001D0120AC27031BC7047B9
S11386900270120A4270120A8270120AC270001D1D
S11386A004C9131B93432B42F2D0E1E701010101FA
S11386B0F0B48AB001216A46D17008900022049275
S11386C06B46DB785B00022423400493049B089CE4
S11386D023606B469970079003926B469B781B014D
S11386E0102423400393039B079C23606B4659701B
S11386F0069002926B465B785B0120242340029330
S1138700029B069C23606B461970059001926B4690
S11387101B789B01402423400193019B059C23600B
S11387200B00040009921D00EDB2ED00082635404F
S11387302560060009920A00D2B2920004273A404A
S113874032600AB0F0BC7047F0B501000025280083
S1138750012213000C001E00F6B2F60180273E40F1
S113876026600B001B68DB091340DBB2002BF8D03A
S11387700B001B685B091340DBB2002B0CD10B0010
S11387801B681B091340DBB2002B05D10B001B68CF
S11387901A40D2B2002A01D007221000C0B2F0BDA4
S11387A0F2B584B004000025280069464870200012
S11387B001260068C0093040C0B2002801D1092058
S11387C04CE02000FFF774FF0D212A00039401956B
S11387D0FF200290039B1700FFB2DB191F7F029B4F
S11387E09F43BC460F00FFB2029B3B4067463B439E
S11387F00193019FBC46039F1300DBB2FB1867463D
S11388001F776B461B7C002B01D0370000E02F0044
S113881069460E700294019505000298694609782C
S11388204018007FA8433900C9B22940014301918F
S1138830019802996A461278891808772000FFF790
S113884083FF6946097C002908D121000968090BC6
S11388500E40F6B2002E01D105210800C0B205B0C9
S1138860F0BD01000A687E4B1A600022CA6170479D
S1138870F3B595B000273800694608707848046855
S113888015988005800D002803D0012069460870E2
S1138890E2E038003D001698854200D3DCE0200079
S11388A001260068C10930000840C0B2002803D185
S11388B0092069460870CFE02000FFF7F9FE052182
S11388C06846017338006A46907114940997FF2032
S11388D01390149A6B469B79D218137F139A93437F
S11388E09C466A46137B139A1A4063461A430992BC
S11388F0099B9C46149B6A4692799A18634613779F
S1138900159A6B46DA7232006B465A7112940897C4
S11389101190129A6B465B79D218137F119A934384
S11389209C466A46D37A119A1A4063461A430892BF
S1138930089B9C46129B6A4652799A1863461377A1
S1138940159AAB02D218120A6B469A7202226B462F
S11389501A71109407970F90109A6B461B79D218CE
S1138960137F0F9A93439C466A46937A0F9A1A4050
S113897063461A430792079B9C46109B6A461279EA
S11389809A1863461377159AAB02D218120C6B46E9
S11389905A7203226B46DA700E9406970D900E9A63
S11389A06B46DB78D218137F0D9A93439C466A4634
S11389B0537A0D9A1A4063461A430692069B9C46C4
S11389C00E9B6A46D2789A1863461377159AAB02BF
S11389D0D218120E6B461A7204226B469A700C94CB
S11389E005970B900C9A6B469B78D218137F0B9AC1
S11389F093439C466A46137A0B9A1A4063461A4379
S1138A000592059B9C460C9B6A4692789A1863468D
S1138A1013776A46D6716A4651700A940497060021
S1138A200A98694649784018007FB0436946C97975
S1138A3031400143049104980A996A46527889188E
S1138A4008772000FFF780FE6946087068460078C2
S1138A50002801D16D1C1EE76846007817B0F0BDF0
S1138A60F0330020F7B598B0002528006946087453
S1138A70824800680090072018990140002901D01D
S1138A800125F6E01A990840002801D00325F0E0FA
S1138A9028006946487201950B95009801270068E3
S1138AA0C10A38000840C0B2012806D1380069461E
S1138AB0487200210098FFF773FE18988005800D16
S1138AC00B900B98A021490544182E001A98864251
S1138AD005D21998805D2070641C761CF6E7009816
S1138AE00068C10938000840C0B2002801D1092536
S1138AF0B7E00098FFF7DCFD06206946C87328003C
S1138B0069460872009817900A95FF2016901799E5
S1138B106A46127A8918097F169A91436A46D37B6A
S1138B20169A1A400A430A920A9A17996B461B7AB4
S1138B30C9180A7718996A4691736946CF710099E2
S1138B4015910995149015996A46D2798918097F67
S1138B50149A91436A46927B149B13400B430993E6
S1138B600999159A6B46DB79D21811771899090A75
S1138B706A46517302216A469171009913910895CE
S1138B80129013996A4692798918097F129A91432F
S1138B906A46527B129B13400B4308930899139A1D
S1138BA06B469B79D21811771899090C6A46117390
S1138BB003216A46517100991191079510901199FA
S1138BC06A4652798918097F109A91436A46127B42
S1138BD0109B13400B4307930799119A6B465B79DB
S1138BE0D21811771899090E6A46D17204216A467F
S1138BF0117100990F9106950E900F996A4612799A
S1138C008918097F0E9A91436A46D27A0E9B1340C3
S1138C100B43069306990F9A6B461B79D21811776A
S1138C201A99C908491E6A469172052700990D913F
S1138C3005950C900D983900C9B24018007F0C9925
S1138C4088436946897A0C9A0A400243059205983A
S1138C500D993A00D2B2891808770098FFF774FD8D
S1138C6005006846407A002803D001210098FFF7E8
S1138C7097FD2800C0B21BB0F0BD0000F033002007
S1138C80F7B596B00026300069468872340016980D
S1138C900721884315908A480568072016990140E2
S1138CA0002901D0012007E118990840002801D0CB
S1138CB0032001E128000068C1090800C007C00FB3
S1138CC0C0B2002801D10920F6E02800FFF7F0FC2B
S1138CD002216846417230006A46D07014950896A5
S1138CE0FF201390149A6B46DB78D218127F139BE3
S1138CF09A436B465F7A139B3B4013430893089B4C
S1138D00149A6F46FF78D2191377169A6B461A7223
S1138D1001226B469A70129507961190129A6B462F
S1138D209B78D218127F119B9A436B461F7A119B32
S1138D303B4013430793079B129A6F46BF78D2199F
S1138D401377169A120A6B46DA716A4651701095B7
S1138D5006960F9010996A4652788918097F0F9ADF
S1138D6091436A46D2790F9B13400B4306930699AD
S1138D70109A6B465B78D21811771699090C6A46DB
S1138D80917103216A4611700E9505960D900E9906
S1138D906A4612788918097F0D9A91436A46927936
S1138DA00D9B13400B43059305990E9A6B461B7854
S1138DB0D21811771699090E6A46517104210C953F
S1138DC004960B900C9A0B00DBB2D218127F0B9B0B
S1138DD09A436B465F790B9B3B4013430493049A7D
S1138DE00C9B0F00FFB2DB191A77189AD208521E97
S1138DF06B461A7105220A95039609900A9B17007F
S1138E00FFB2DB191F7F099B9F43BC466B461F794A
S1138E10099B3B4067463B430393039FBC460A9F21
S1138E201300DBB2FB1867461F773400082C1ED2F0
S1138E3001002200521D039500960190039B170028
S1138E40FFB2DB191F7F019B9F43BC460F00FFB29B
S1138E50019B3B4067463B430093009FBC46039FF6
S1138E601300DBB2FB1867461F77641CDEE728009B
S1138E70FFF76AFC290001200968CA0801001140B3
S1138E80C9B2012906D02900096889080840C0B27E
S1138E90012801D1062000E030000100C9B20029F8
S1138EA00AD1340018998C4206D216990919097806
S1138EB0179A1155641CF5E7C0B219B0F0BD000053
S1138EC0F0330020002202604160012303724272E9
S1138ED0704770B504000E001500B548215A95205E
S1138EE0C0002018FFF7EEFF7820205C012806D090
S1138EF02A0092B2310020001830FCF74BFB70BD01
S1138F00FEB505000E001400082100226F4638004B
S1138F10FCF704F92000C0B2782806D0A448295AE6
S1138F209520C0002818FFF7CDFF7920285C002881
S1138F3014D02000C0B211280FD02000C0B21228D3
S1138F400BD02000C0B2312807D02000C0B27E2848
S1138F5003D02000C0B27F2800D10AE068467F21F8
S1138F600170467084700322694628001830FCF7AB
S1138F7011FBF7BD30B500200300042102001300EB
S1138F800C00DBB2E4B2A34208D28A4B1400E4B270
S1138F9014256C431B191871521CF0E730BD70B5D1
S1138FA000210C0004220B001C001500E4B2EDB2F9
S1138FB0AC4212D27F4C1D00EDB214267543655BA2
S1138FC00600B6B2B54206D11D00EDB214267543B3
S1138FD06419217101E05B1CE6E770BDFEB5040075
S1138FE00F001500089E3088002C06D1390089B284
S1138FF0002902D0002131800CE00021020092B24D
S1139000A954401C694608806846008830806A4834
S1139010FFF7C5FFF7BD70477047FFB581B0070084
S113902000252E002C0028006946087029002A001B
S1139030002F02D10A98058039E004206B4618708D
S11390406B465870280001006A461278C9B29142F2
S11390500BD20100C9B2791849780322121AD2003E
S1139060914031430E00401CEDE7280069464978E1
S1139070C0B288420BD22800C0B23818407903210C
S1139080491BC9008840204304006D1CEDE7210002
S11390903000FEF767FB7F200399087031200399A5
S11390A0487078200399887003200A99088005B0D5
S11390B0F0BD70477047FFB581B00024270026003B
S11390C02500200021000A9A118021000800C0B266
S11390D004280BDA01980A00D2B2805C0322521AE7
S11390E0D200904038430700491CEFE720000100FC
S11390F0C9B204290CDA01990200D2B2891809799B
S11391000322121AD200914031430E00401CEEE7B4
S11391102000C0B204280CDA01982100C9B240181A
S1139120007A0321091BC900884028430500641CF8
S1139130EEE72A0031003800FEF796FB05B0F0BDDB
S113914070477047FBB504001700089D2E88FEF792
S1139150D8FA012825D10020C043C2490968C24A6F
S1139160914208D3E0229202914204D20A1F009253
S1139170009A12681000BD4A1268BD4B9A4209D089
S1139180BC4A904206D0012233009BB2FA54761CAA
S11391902E800CE0002233009BB2FA54761C2E8001
S11391A005E00220310089B27854761C2E80F7BD88
S11391B08C040000AC0800200302000070477047D4
S11391C0F7B5FFB087B000260496300069460873EF
S11391D03000694648813400300069460870042034
S11391E069464873802080000190320005AD0199E2
S11391F02800FBF793FF30006946088188A800889F
S113920086998968869A7A23D25C120189184978EA
S113921089B2884205D2132231218698FFF770FE65
S11392201CE17F27879840783840694608738798FF
S1139230807800028799C97840186946C88188A84F
S11392400088001F6946488168464089002802D08A
S11392508798001D0490350028006946497BC0B2F8
S1139260884234D284482900C9B214225143415A55
S11392706A46D289914228D1869949782A00D2B285
S113928014235A4382189278114218D02900C9B283
S1139290142251434118C97800290FD02900C9B2BA
S11392A0142251434018C07886998978884205D0A1
S11392B0332231218698FFF723FECFE007E02222F4
S11392C031218698FFF71CFEC8E06D1CC4E7280016
S11392D06946497BC0B2884205D331223121869840
S11392E0FFF70EFEBAE0802080000190009605ACE6
S11392F0009A01992000FBF711FF05AC7120207042
S113930087984078607087988078A0708798C07834
S1139310E0700420694608816846007B012804D077
S113932079D3032853D024D375E0534E2800C0B218
S11393301421484330180079012808D127703120BE
S113934060702420A07003206946088110E002A800
S1139350009080239B0005AA684641890498B4467E
S11393602F00FFB2142677436646F619B668B04755
S11393705AE041482900C9B21422514340180079E7
S113938000281BD002A8009080239B0005AA6846F1
S1139390418904980190384884462F00FFB2142074
S11393A047436046C019C7680198B8473248290046
S11393B0C9B2142251434018067107E027703120C6
S11393C060702420A0700320694608812CE02A4E96
S11393D02800C0B21421484330180079002811D065
S11393E002A8009080239B0005AA6846418904983E
S11393F0B4462F00FFB2142677436646F619366941
S1139400B04707E02770312060702420A07003204B
S11394106946088108E02770312060701220A0702E
S113942003206946088119E068460089042809DB9D
S11394302078712806D16846028905A98698FFF725
S113944048FD0BE068460089032807D120787F286F
S113945004D1A27831218698FFF752FD7FB00AB07B
S1139460F0BD0000F87F030001000100C00001000E
S1139470DDCCBBAAAABBCCDDAC0800200022026074
S11394804160012303724272704770B504000E00FC
S113949015009748215A9520C0002018FFF7EEFFC9
S11394A07820205C012806D02A0092B231002000E6
S11394B01830FCF76FF870BDFEB505000E001400FF
S11394C0082100226F463800FBF728FE2000C0B2B6
S11394D0782806D08648295A9520C0002818FFF716
S11394E0CDFF7920285C002814D02000C0B21128B8
S11394F00FD02000C0B212280BD02000C0B23128F7
S113950007D02000C0B27E2803D02000C0B27F283C
S113951000D10AE068467F210170467084700322FE
S1139520694628001830FCF735F8F7BDFAB583B062
S11395300400150001A86F490A6802609020C00069
S1139540201803C8009001A8009901700099090A25
S113955041700099090CC9B2427807235A4389180B
S113956081700099090EC9B2027803235A438918FD
S1139570C1706846007C042819D3042001000A9AAB
S113958011806946097BA278914208D10290002695
S11395902F00320002993800FBF7C0FD07E002906B
S11395A001AE2F00029A31003800FBF7A9FD05B087
S11395B0F0BDFEB504002000C0B2012802D0092885
S11395C046D093E04C4D68460E782F78774007706C
S11395D04E786F78774047708E78AF787740877091
S11395E0CE78ED787540C57001ADC678F027374068
S11395F02F70C678B700BC263E404778BF07BF0F20
S113960037436F7046783700FFB2BF08BC4607780F
S1139610C0263E4067463E43AE70067836018078E9
S11396200007000F3043E87028781E78B0420BD151
S113963068785E78B04207D1A8789E78B04203D1AA
S1139640E878DD78A84201D0002050E001204EE007
S1139650294D68460E782F78774007704E786F78DA
S1139660774047708E78AF7877408770CE78ED7802
S11396707540C57001AD4678B700BC468778F026C2
S11396803E4067463E432E700678F6B2B6083B2746
S11396903740BC4647787E263E4067463E436E7060
S11396A0C6783700FFB23F09BC4607782C263E40F7
S11396B067463E43AE7086783601C0787D27074002
S11396C03743EF7028781E78B0420BD168785E7803
S11396D0B04207D1A8789E78B04203D1E878DD780B
S11396E0A84201D0002002E0012000E00020FEBDDD
S11396F08C0400000CBD000010BD0000F7B586B05E
S113970000206946887208210020009003AC009A6A
S11397102000FBF703FD00206946C880002069464D
S113972008810020694648716846008C069989685A
S1139730069A7A23D25C12018918497889B2884240
S113974005D2132227210698FFF7B6FE14E10698E6
S11397504078012805D1222227210698FFF7ACFE84
S11397600AE1079840784006400E6946087103AF45
S11397706720387068460079787068460079C007B9
S113978000D47FE0002630007C49087034002000BB
S1139790C0B2022837DA7A4D684600792100C9B28E
S11397A00901695C88422CD12000C0B2000128184C
S11397B080782100C9B209016918497888421FD20A
S11397C006989021C90040180CC808382000C0B27F
S11397D000012818083003C8121A8B416948002177
S11397E08B4208DC01DB824205D23622272106980F
S11397F0FFF762FEC0E02000C0B2000128184670E6
S113980001E0641CC3E72000C0B2022805DB31225A
S113981027210698FFF750FEAEE00620694608812E
S113982001A8801C009068460389DBB2BA1C684614
S113983001790698FFF77AFE6846C08800281BD095
S11398406846C288921C92B203A90698FFF71DFECF
S113985068460079494908706846C0884A490880C2
S11398606846C088009003A8851C484E009A2900C9
S11398703000FBF745FC7FE0312227210698FFF7F3
S11398801BFE79E03D4D684600792978491C8842E1
S113989005D0242227210698FFF70EFE6CE06846C7
S11398A0008C801E80B200900798831C3648028882
S11398B036492878FFF77DFE694648716846407945
S11398C0012822D1022203A90698FFF7DEFD002019
S11398D00100297069460979491E069A91700400AD
S11398E02100C9B2022947DA25496A4612792300C0
S11398F0DBB21B01CB5C9A4205D102002300DBB230
S11399001B01C9184A70641CEAE73522272106980E
S1139910FFF7D2FD00242000C0B202282CDA184A36
S113992028782100C9B20901515C884222D1200063
S1139930C0B2000110184078401C2100C9B20901CE
S1139940511848702000C0B200011018807821001E
S1139950C9B209015118497888420BD2069890215E
S1139960C900401803C82300DBB21B01D218083217
S113997003C2083A641CCEE709B0F0BD082E0020EB
S11399801808002010270000042E0020B82D002005
S113999000000000963007772C610EEEBA51099949
S11399A019C46D078FF46A7035A563E9A395649EA5
S11399B03288DB0EA4B8DC791EE9D5E088D9D297C9
S11399C02B4CB609BD7CB17E072DB8E7911DBF9025
S11399D06410B71DF220B06A4871B9F3DE41BE8449
S11399E07DD4DA1AEBE4DD6D51B5D4F4C785D383A5
S11399F056986C13C0A86B647AF962FDECC9658A49
S1139A004F5C0114D96C0663633D0FFAF50D088DA4
S1139A10C8206E3B5E10694CE44160D5727167A248
S1139A20D1E4033C47D4044BFD850DD26BB50AA5A4
S1139A30FAA8B5356C98B242D6C9BBDB40F9BCACC8
S1139A40E36CD832755CDF45CF0DD6DC593DD1AB24
S1139A50AC30D9263A00DE518051D7C81661D0BF48
S1139A60B5F4B42123C4B3569995BACF0FA5BDB8A4
S1139A709EB802280888055FB2D90CC624E90BB148
S1139A80877C6F2F114C6858AB1D61C13D2D66B6A4
S1139A909041DC760671DB01BC20D2982A10D5EF08
S1139AA08985B1711FB5B606A5E4BF9F33D4B8E864
S1139AB0A2C9077834F9000F8EA8099618980EE108
S1139AC0BB0D6A7F2D3D6D08976C6491015C63E664
S1139AD0F4516B6B62616C1CD83065854E0062F288
S1139AE0ED95066C7BA5011BC1F4088257C40FF5E4
S1139AF0C6D9B06550E9B712EAB8BE8B7C88B9FC08
S1139B00DF1DDD62492DDA15F37CD38C654CD4FB63
S1139B105861B24DCE51B53A7400BCA3E230BBD407
S1139B2041A5DF4AD795D83D6DC4D1A4FBF4D6D363
S1139B306AE96943FCD96E34468867ADD0B860DA07
S1139B40732D0444E51D03335F4C0AAAC97C0DDD63
S1139B503C710550AA41022710100BBE86200CC987
S1139B6025B56857B3856F2009D466B99FE461CEE3
S1139B700EF9DE5E98C9D9292298D0B0B4A8D7C707
S1139B80173DB359810DB42E3B5CBDB7AD6CBAC063
S1139B902083B8EDB6B3BF9A0CE2B6039AD2B1747F
S1139BA03947D5EAAF77D29D1526DB048316DC73DB
S1139BB0120B63E3843B64943E6A6D0DA85A6A7A7F
S1139BC00BCF0EE49DFF099327AE000AB19E077DDB
S1139BD044930FF0D2A3088768F2011EFEC20669FF
S1139BE05D5762F7CB67658071366C19E7066B6E5B
S1139BF0761BD4FEE02BD3895A7ADA10CC4ADD677F
S1139C006FDFB9F9F9EFBE8E43BEB717D58EB060DA
S1139C10E8A3D6D67E93D1A1C4C2D83852F2DF4F7E
S1139C20F167BBD16757BCA6DD06B53F4B36B248DA
S1139C30DA2B0DD84C1B0AAFF64A0336607A04417E
S1139C40C3EF60DF55DF67A8EF8E6E3179BE6946DA
S1139C508CB361CB1A8366BCA0D26F2536E26852FE
S1139C6095770CCC03470BBBB91602222F2605555A
S1139C70BE3BBAC5280BBDB2925AB42B046AB35C7E
S1139C80A7FFD7C231CFD0B58B9ED92C1DAEDE5BDA
S1139C90B0C2649B26F263EC9CA36A750A936D02BE
S1139CA0A906099C3F360EEB85670772135700051A
S1139CB0824ABF95147AB8E2AE2BB17B381BB60C3E
S1139CC09B8ED2920DBED5E5B7EFDC7C21DFDB0B9A
S1139CD0D4D2D38642E2D4F1F8B3DD686E83DA1FBE
S1139CE0CD16BE815B26B9F6E177B06F7747B7181A
S1139CF0E65A0888706A0FFFCA3B06665C0B0111BE
S1139D00FF9E658F69AE62F8D3FF6B6145CF6C1619
S1139D1078E20AA0EED20DD75483044EC2B30339BD
S1139D20612667A7F71660D04D476949DB776E3E19
S1139D304A6AD1AEDC5AD6D9660BDF40F03BD8373D
S1139D4053AEBCA9C59EBBDE7FCFB247E9FFB53099
S1139D501CF2BDBD8AC2BACA3093B353A6A3B424BD
S1139D600536D0BA9306D7CD2957DE54BF67D92319
S1139D702E7A66B3B84A61C4021B685D942B6F2ABD
S1139D8037BE0BB4A18E0CC31BDF055A8DEF022D19
S1139D90F0B592B00123180069468870E149049136
S1139DA00498C06A0422D24310406C46A478A400EC
S1139DB004252C4004430E940E98049CE062180081
S1139DC06C46607003910398C06A0124A0436C46FA
S1139DD064781C4004430D940D98039CE0620020B9
S1139DE004006D462C7002910299C96A0A406946C2
S1139DF0097889000424214011430C910C99029A9A
S1139E00D162CD490B91CD490A910B9A0A9C2266E5
S1139E10CB4A0992CB4A0892099A089C8025625140
S1139E20C94CCA4A0792079A802554511D00C84A52
S1139E300192019A12680F26B2432E00F6B2360739
S1139E40360F16430696069A019E3260C14A059261
S1139E50059E3668360EB607B60FF6B2022E2DD121
S1139E6004006D462C70BC4C6668BC4D35406E4693
S1139E7036783702F02636013E402E430396039D82
S1139E80656005000292029E3768B54E3E40019619
S1139E90019FBC462E00F6B23704C026B6023E40EF
S1139EA067463E430196019E029F3E60140024686B
S1139EB0240EA407A40FE4B2002CF7D11C000191D6
S1139EC0019DED680C26B5432600F6B2B7000C26BA
S1139ED03E402E430296029D019EF5601D000091B6
S1139EE0009EF6680127BE432F00FFB21F40374390
S1139EF0009EF7600C00246AA5081C002C40E4B204
S1139F00002CF7D004006D46EC71904C0994099C28
S1139F10A568944C2C406D46ED792D04802676027C
S1139F20354025431195119C099DAC6004006D4694
S1139F30AC710891089C64690125AC436D46AD7908
S1139F401D4025431095109C089D6C611C006D46B6
S1139F506C710791079CA4691025AC436D466D791B
S1139F602D011026354025430F950F9C079DAC61AC
S1139F7004006D462C710691069C65697A4C2C4050
S1139F806D462D792D02C026B6002E4026430E962E
S1139F900E9C069D6C6128246D46EC700591059C11
S1139FA06469FE25AC436D46ED786D00FE262E40B7
S1139FB026430D960D9C059D6C611C006D46AC708E
S1139FC00491049C6569694C2C406D46AD78AD06DE
S1139FD08026F604354025430C950C9C049D6C6149
S1139FE002246D466C700391039C6569604C2C409F
S1139FF06D466D78ED02E026B6012E4026430B96A1
S113A0000B9C039D6C611C006D462C700291029C9C
S113A01064690125AC436D462D781D4025430A959E
S113A0200A9C029D6C61FA246401524D2C60524CCE
S113A0302060524D05262E602E6880277F02BE4286
S113A040FAD304262E604B4D286020600C00256A4C
S113A0501C002C40E4B2002CF8D06C4663703E4BDC
S113A0605D683E4C25400295F0252D01029E6F4609
S113A0707F783F022F4037430297029E5E6002269C
S113A0806F463E700392039E3768354E3E400196FC
S113A090019FBC466E4636783704C026B6023E4061
S113A0A067463E430196019E039F3E6013001B6872
S113A0B01B0E9B079B0FDBB2022BF7D103006E46EE
S113A0C03370234B0293029B1B680F26B3436E46E7
S113A0D036783607360F1E430796079B029E336079
S113A0E003000192019A126822401E00F6B2360261
S113A0F02E4016430696069A019E32600922204E8F
S113A100C827F7593C401700FFB23F023D402543A2
S113A110C8243551059004910599049C2166039047
S113A120084901E000F00540039C8027CC51074C0E
S113A1308027E05112B0F0BD2020961900E00640BF
S113A1405245535500F006404B4D435200F0074032
S113A15000E4064000E8064000000240FFF0FFFF74
S113A160FFFFFCFFFFFFFEFFFFFCFFFFFFFFFFFB06
S113A170FFC7FFFF14E000E018E000E010E000E09B
S113A18000F806400022026041600123037242721B
S113A190704770B504000E001500B948215A952087
S113A1A0C0002018FFF7EEFF7820205C012806D0BD
S113A1B02A0092B2310020001830FBF7EBF970BD91
S113A1C0FEB505000E001400082100226F46380079
S113A1D0FAF7A4FF2000C0B2782806D0A848295A6C
S113A1E09520C0002818FFF7CDFF7920285C0028AF
S113A1F014D02000C0B211280FD02000C0B2122801
S113A2000BD02000C0B2312807D02000C0B27E2875
S113A21003D02000C0B27F2800D10AE068467F2125
S113A2200170467084700322694628001830FBF7D9
S113A230B1F9F7BDF7B5FFB085B005000020694658
S113A240488000206946C88000260020694688802E
S113A25000240020694608708021890000200290B3
S113A26004AF029A3800FAF759FF86A80088A96853
S113A2707A22AA5C12018918497889B2884205D2E7
S113A280132222212800FFF79BFFF6E086A800880E
S113A290401EC00705D5132222212800FFF790FF96
S113A2A0EBE086A8008840086946488068464088F4
S113A2B0002805D1132222212800FFF781FFDCE0CA
S113A2C0622004A9320092B28854761C0127380017
S113A2D086A9098880B2884200D3BEE085983900F7
S113A2E089B2405C000285993A0092B28918497893
S113A2F008436946C880002001006A4611700400C2
S113A3002000A98A80B2884200D3A0E028692100F5
S113A31089B214224A43805A6946C988884200D0C7
S113A32093E0A8782969220092B214235343C918F0
S113A3300979884205D0332222212800FFF740FF03
S113A3409BE0300080B22969220092B21423534367
S113A350C91889894018801C4A49884205DB14229F
S113A36022212800FFF72CFF87E02869210089B209
S113A37014224A4380188078052809D0687829690E
S113A380220092B214235343C918C978884205D2D3
S113A390222222212800FFF713FF6EE02869210002
S113A3A089B214224A4380188289D2B228692100D2
S113A3B089B214234B43C0188168280005002B6917
S113A3C09C4623009BB21420584363461818036923
S113A3D02800984701206946087004A885993A0026
S113A3E092B2895C320092B28154761C85993A000B
S113A3F092B289184978320092B28154761C684628
S113A40086802869210089B214224A4380188089F1
S113A41003902869210089B214224A438018806875
S113A420029004A8694689884618039A0299300064
S113A430FAF766FE684680882969220092B21423DE
S113A4405343C9188989461801E0641C58E76846D3
S113A4500078002801D0BF1C39E76846007800283E
S113A46006D0320092B204A92800FFF792FE04E05D
S113A470312222212800FFF7A3FE7FB008B0F0BDEF
S113A4808C040000010200000022026041600123EC
S113A49003724272704770B504000E00150026481E
S113A4A0215A9520C0002018FFF7EEFF7820205C89
S113A4B0012806D02A0092B2310020001830FBF7A0
S113A4C069F870BDFEB505000E00140008210022D5
S113A4D06F463800FAF722FE2000C0B2782806D072
S113A4E01548295A9520C0002818FFF7CDFF792078
S113A4F0285C002814D02000C0B211280FD02000FE
S113A500C0B212280BD02000C0B2312807D02000DE
S113A510C0B27E2803D02000C0B27F2800D10AE058
S113A52068467F21017046708470032269462800C2
S113A5301830FBF72FF8F7BD8C04000010B5002489
S113A540FCF760FE801C10BD10B501000020030064
S113A55001221300DBB2052B0CDA04239B1ADB0067
S113A5600C00DC40002C03D005239B1A180001E0EA
S113A570521CEEE7C0B210BDF7B586B000273E000E
S113A5803800694608703D00380069468870380014
S113A59069464870029738006946C87038006946B1
S113A5A0888008213A0003AC2000FAF7B7FD06982A
S113A5B04078012805D1222234210698FFF782FF32
S113A5C0A3E06846008C06998968069A7A23D25CCF
S113A5D012018918497889B2884205D2132234219C
S113A5E00698FFF76FFF90E0079880780007000F48
S113A5F06946087007988078C0B200096946887077
S113A6006846007800280BD068460078052807D2F1
S113A61068468078002803D068468078052805D3EA
S113A620312234210698FFF74DFF6EE03800010017
S113A6306A461278C9B2914208D23102079A0300DD
S113A640DBB2D218D2788E18401CF0E73800694685
S113A6508978C0B288420BD2280207996A461278D8
S113A6603B00DBB2D2188918C97845187F1CEDE786
S113A670002D05D1222234210698FFF723FF44E060
S113A68000F087F8300000F092F8280000F092F80B
S113A690012000F095F8FFF751FF02900298FFF7B0
S113A6A053FF6946487003A874216A46928881540E
S113A6B069468988491C6A46527812010B009BB28C
S113A6C0C254491C6A469180012469464978220093
S113A6D0D2B291420FD302996A465278121BD20029
S113A6E0D1406A469288815469468988491C6A46E1
S113A6F09180641CE9E729003000FDF75FF86846A3
S113A700828803A90698FFF7C6FE09B0F0BD0000D1
S113A7100022026041600123037242727047FEB559
S113A72005000E001400082100226F463800FAF7D5
S113A730F5FC2000C0B2782806D06B48295A952031
S113A740C0002818FFF7E4FF7920285C002814D003
S113A7502000C0B211280FD02000C0B212280BD0A4
S113A7602000C0B2312807D02000C0B27E2803D018
S113A7702000C0B27F2800D10AE068467F21017022
S113A780467084700322694628001830FAF702FFE5
S113A790F7BD00200100554A11700100544A1170A0
S113A7A05449086054490860544908607047524944
S113A7B00860704751490860704750480068704706
S113A7C04F49087070474E48007870474948006800
S113A7D07047F7B5040000206946087060780128C6
S113A7E005D1222236212000FFF799FF79E068463F
S113A7F00089A1687A22A25C12018918497889B279
S113A800884205D2132236212000FFF788FF68E032
S113A8103B480078012802D0022857D05CE0334D31
S113A820019840782870324E2878317888420BD0CD
S113A83028783178491CC9B2884205D07322362160
S113A8402000FFF76CFF4CE02A4F2C480068396861
S113A8506A4612898918891E884205D271223621D6
S113A8602000FFF75CFF3CE0FCF7DAFC6946087067
S113A8706846007800280FD068460078012805D182
S113A880932236212000FFF74AFF04E0922236216A
S113A8902000FFF744FF24E028783178491CC9B22E
S113A8A0884212D12A7868460189891E89B20198A2
S113A8B0801CFCF7ACFF012805D13868694609897A
S113A8C04018801E3860287830700AE03122362122
S113A8D02000FFF724FF04E0242236212000FFF7A4
S113A8E01EFFF7BD000000008C0400000B2E0020AA
S113A8F00C2E0020C82D0020C02D0020C42D0020C7
S113A9000A2E002000220260416001230372427279
S113A910704770B504000E0015007F48215A952039
S113A920C0002018FFF7EEFF7820205C012806D035
S113A9302A0092B2310020001830FAF72BFE70BDC5
S113A940FEB505000E001400082100226F463800F1
S113A950FAF7E4FB2000C0B2782806D06E48295AE2
S113A9609520C0002818FFF7CDFF7920285C002827
S113A97014D02000C0B211280FD02000C0B2122879
S113A9800BD02000C0B2312807D02000C0B27E28EE
S113A99003D02000C0B27F2800D10AE068467F219E
S113A9A00170467084700322694628001830FAF753
S113A9B0F1FDF7BDF6B583B004000E0008210027B1
S113A9C03A0001AD2800FAF7A9FB3800694648703F
S113A9D06846008AA1687A22A25C12018918497823
S113A9E089B2884205D2132228212000FFF7A8FF4C
S113A9F08EE06078012805D1222228212000FFF76B
S113AA009FFF85E070784006400E69460870B5786F
S113AA1001A8682101706946097841706846007888
S113AA20002805D0022838D01CD3032850D06AE06F
S113AA302800C0B2012807D02800C0B2022803D0E1
S113AA402800C0B2032807D134480770022201A9A4
S113AA502000FFF75EFF04E0312228212000FFF7E9
S113AA606FFF55E02800C0B2012807D02800C0B20B
S113AA70022803D02800C0B2032808D101202749A6
S113AA800870022201A92000FFF743FF04E03122ED
S113AA9028212000FFF754FF3AE02800C0B2012823
S113AAA007D02800C0B2022803D02800C0B203286F
S113AAB008D1022019490870022201A92000FFF7D9
S113AAC028FF04E0312228212000FFF739FF1FE08E
S113AAD02800C0B2012807D02800C0B2022803D041
S113AAE02800C0B2032808D103200C4908700222B0
S113AAF001A92000FFF70DFF04E0312228212000E6
S113AB00FFF71EFF04E0122228212000FFF718FFA0
S113AB1005B0F0BD000000008C040000092E0020E8
S113AB20002202604160012303724272704770B5D3
S113AB3004000E0015002648215A9520C000201854
S113AB40FFF7EEFF7820205C012806D02A0092B29D
S113AB50310020001830FAF71DFD70BDFEB5050068
S113AB600E001400082100226F463800FAF7D6FAC6
S113AB702000C0B2782806D01548295A9520C00074
S113AB802818FFF7CDFF7920285C002814D0200076
S113AB90C0B211280FD02000C0B212280BD0200060
S113ABA0C0B2312807D02000C0B27E2803D02000D4
S113ABB0C0B27F2800D10AE068467F210170467048
S113ABC084700322694628001830FAF7E3FCF7BDC5
S113ABD08C040000F6B585B005000E0000242000AA
S113ABE0694608802000694648800821220003AF96
S113ABF03800FAF793FA6846008BA9687A22AA5CAF
S113AC0012018918497889B2884205D213222E216B
S113AC102800FFF7A3FF82E070780002B1780843B0
S113AC206946088003A86E21017071784170B1787B
S113AC3081702000A98A80B288426BD228692100E1
S113AC4089B214224A43805A6946098888425FD1EE
S113AC502869210089B214224A4380180079002807
S113AC600FD0A8782969220092B214235343C9183B
S113AC700979884205D0332222212800FFF76EFF8C
S113AC804DE06846008BC01E2969220092B214234D
S113AC905343C9188989884205D013222E212800DC
S113ACA0FFF75CFF3BE02869210089B214224A4384
S113ACB080188078032809D068782969220092B224
S113ACC014235343C918C978884205D222222E215D
S113ACD02800FFF743FF22E02869210089B21422EB
S113ACE04A43801880890290F01C01902869210051
S113ACF089B214224A4380188768029A019938005D
S113AD00FAF7FEF9032203A92800FFF710FF06E073
S113AD10641C8EE731222E212800FFF71FFF07B0A5
S113AD20F0BD000000220260416001230372427200
S113AD30704770B504000E0015006A48215A95202A
S113AD40C0002018FFF7EEFF7820205C012806D011
S113AD502A0092B2310020001830FAF71BFC70BDB3
S113AD60FEB505000E001400082100226F463800CD
S113AD70FAF7D4F92000C0B2782806D05948295AE5
S113AD809520C0002818FFF7CDFF7920285C002803
S113AD9014D02000C0B211280FD02000C0B2122855
S113ADA00BD02000C0B2312807D02000C0B27E28CA
S113ADB003D02000C0B27F2800D10AE068467F217A
S113ADC00170467084700322694628001830FAF72F
S113ADD0E1FBF7BDF2B582B004001600082100279C
S113ADE03A006D462800FAF799F93000A1687A22F2
S113ADF0A25C12018918497880B289B2884205D0D0
S113AE00132210212000FFF7ABFF69E0029840787D
S113AE1045066D0E68465021017045709121C900A8
S113AE20615A89B2090A81709121C900615AC170BD
S113AE302D49615A89B2090A01712B49615A41713C
S113AE402800C0B2012806D045D303280DD01DD355
S113AE5004282FD03FE0A7706570062269462000C1
S113AE60FFF767FFFEF786F83AE0A77065700622E1
S113AE7069462000FFF75DFFFEF77CF81948215A68
S113AE809520C0002018FFF74DFF29E0A7706570DA
S113AE90062269462000FFF74CFF1248215A9520EC
S113AEA0C0002018FFF73EFFFEF764F80120FCF70E
S113AEB033FC15E0A7706570062269462000FFF791
S113AEC038FFFEF757F80748215A9520C00020188C
S113AED0FFF728FF04E0122210212000FFF740FFB3
S113AEE0F7BD00008C0400008A040000010100008A
S113AEF02D0100000D020000000000002F020000E0
S113AF0021030000CB04000021050000F10500002E
S113AF1047060000190700006F0700003D08000005
S113AF20930800005D090000B30900007D0A0000D9
S113AF30D30A0000A10B0000FB0B00005D0C000015
S113AF40950C0000C50C0000FF0C0000330D000040
S113AF50970D0000250E00007B0F0000E512000095
S113AF6000000000EF120000131300003D13000066
S113AF70611300008B130000000000009713000011
S113AF80251400004F14000079140000A3140000DD
S113AF90CD140000F7140000211500004B1500002B
S113AFA019160000A7170000131800001519000057
S113AFB085190000651A0000A71A0000F31A0000A2
S113AFC0351B0000851B0000C71B0000191C000076
S113AFD0591C0000AD1C0000D31C0000FD1C000027
S113AFE0231D00004D1D0000731D00009D1D000069
S113AFF0C31D0000ED1D0000131E00003D1E0000D7
S113B000631E00008D1E00001B1F00003D20000079
S113B010632000008D200000F12000009921000031
S113B020FD210000A522000009230000AB2300003D
S113B0300F240000B524000019250000C1250000DC
S113B040E7250000112600003726000061260000D5
S113B05089260000B7260000DF2600000D27000027
S113B06035270000632700008B270000B927000064
S113B07000000000C327000000000000CD270000EE
S113B08000000000D7270000552800003F290000D9
S113B090BD290000A72A0000E12A00003D2B000082
S113B0A0772B0000CF2B0000F72B0000002202605A
S113B0B04160012303724272704770B504000E00B0
S113B0C015002648215A9520C0002018FFF7EEFFEE
S113B0D07820205C012806D02A0092B2310020009A
S113B0E01830FAF757FA70BDFEB505000E001400CB
S113B0F0082100226F463800FAF710F82000C0B289
S113B100782806D01548295A9520C0002818FFF73A
S113B110CDFF7920285C002814D02000C0B211286B
S113B1200FD02000C0B212280BD02000C0B23128AA
S113B13007D02000C0B27E2803D02000C0B27F28F0
S113B14000D10AE068467F210170467084700322B2
S113B150694628001830FAF71DFAF7BD8C04000080
S113B160F2B582B0040016000022150008216F46D3
S113B1703800F9F7D3FF6078012805D1222237215E
S113B1802000FFF7B1FF40E03000A1687A22A25C02
S113B19012018918497880B289B2884205D21322F3
S113B1A037212000FFF7A0FF2FE0772069462A000F
S113B1B092B288546D1C2F00FFF705FB012802D0C2
S113B1C0022814D019E0FFF701FB0500FFF7F5FA98
S113B1D0854205D0132237212000FFF785FF11E0B7
S113B1E03A0092B269462000FFF767FF0AE0312275
S113B1F037212000FFF778FF04E0242237212000C4
S113B200FFF772FF0020FFF7DBFAF7BD00220260B0
S113B2104160012303724272704770B504000E004E
S113B22015002648215A9520C0002018FFF7EEFF8C
S113B2307820205C012806D02A0092B23100200038
S113B2401830FAF7A7F970BDFEB505000E0014001A
S113B250082100226F463800F9F760FF2000C0B2D1
S113B260782806D01548295A9520C0002818FFF7D9
S113B270CDFF7920285C002814D02000C0B211280A
S113B2800FD02000C0B212280BD02000C0B2312849
S113B29007D02000C0B27E2803D02000C0B27F288F
S113B2A000D10AE068467F21017046708470032251
S113B2B0694628001830FAF76DF9F7BD8C040000D0
S113B2C0FEB504000F0016000821002201AD28007D
S113B2D0F9F724FFFF253100A0687A22A25C12014D
S113B2E08018407889B280B2814205D0132211219E
S113B2F02000FFF7A9FF37E078784006400E694642
S113B300087001A85121017069460978417085705F
S113B31068460078012804D021D3032815D00AD325
S113B3201DE0022201A92000FFF777FF012101207F
S113B330FCF708FA18E0022201A92000FFF76DFFCC
S113B34002210120FCF7FEF90EE0022201A92000EF
S113B350FFF763FF03210120FCF7F4F904E0122254
S113B36011212000FFF770FFF7BD00000100050068
S113B37000000000000000000000000009000500BB
S113B3800000000000000000000000003372000014
S113B390817200006D730000957600005574000002
S113B3A0497600000100000032070000DF070000BA
S113B3B0B20700009C200020000200009C22002014
S113B3C00204000000000000495E0000EB5C000085
S113B3D03200F4018813000027C08FD2A0D34DDCC3
S113B3E0FF000000000000000000FFFF00FFFEFF60
S113B3F0FFFFFFFFFFFFFFFFFEFFFFFFFFFFFFFF5A
S113B40000FF0209000000001B900000B390000040
S113B410B59000000302030000000000DD8F00006F
S113B42017900000199000000202020900000000B9
S113B430B7900000419100004391000001FF020910
S113B4400000000045910000BD910000BF91000084
S113B45086F1060100000000CC2D00200100000050
S113B4606771000087F1060100000000CD2D002067
S113B470080000006D71000080F10601000000006A
S113B480D52D0020080000004971000091F106014B
S113B49000000000DD2D0020180000008D71000068
S113B4A093F1060100000000F52D002004000000C7
S113B4B0C971000095F1060100000000F92D00207B
S113B4C008000000E57100000022026041600123D1
S113B4D003724272704770B504000E0015002648CE
S113B4E0215A9520C0002018FFF7EEFF7820205C39
S113B4F0012806D02A0092B2310020001830FAF751
S113B50049F870BDFEB505000E00140008210022A4
S113B5106F463800F9F702FE2000C0B2782806D042
S113B5201548295A9520C0002818FFF7CDFF792027
S113B530285C002814D02000C0B211280FD02000AD
S113B540C0B212280BD02000C0B2312807D020008E
S113B550C0B27E2803D02000C0B27F2800D10AE008
S113B56068467F2101704670847003226946280072
S113B5701830FAF70FF8F7BD8C040000FEB504008C
S113B5800E001500082100226F463800F9F7C6FDA9
S113B5902800A1687A22A25C12018918497880B235
S113B5A089B2884205D2132285212000FFF7AAFF21
S113B5B02DE06078012805D1222285212000FFF7A3
S113B5C0A1FF24E0707847067F0E6846C52101700C
S113B5D047703800C0B2012802D0022809D011E017
S113B5E0012000F015F8022269462000FFF773FFDE
S113B5F00DE0002000F00CF8022269462000FFF75D
S113B6006AFF04E0122285212000FFF77BFFF7BDCB
S113B6100149087070470000072E002000220260D4
S113B6204160012303724272704770B504000E003A
S113B63015002648215A9520C0002018FFF7EEFF78
S113B6407820205C012806D02A0092B23100200024
S113B6501830F9F79FFF70BDFEB505000E00140009
S113B660082100226F463800F9F758FD2000C0B2C7
S113B670782806D01548295A9520C0002818FFF7C5
S113B680CDFF7920285C002814D02000C0B21128F6
S113B6900FD02000C0B212280BD02000C0B2312835
S113B6A007D02000C0B27E2803D02000C0B27F287B
S113B6B000D10AE068467F2101704670847003223D
S113B6C0694628001830F9F765FFF7BD8C040000BF
S113B6D0FEB504000E001500082100226F46380054
S113B6E0F9F71CFD2800A1687A22A25C12018918CE
S113B6F0497880B289B2884205D013223E212000C5
S113B700FFF7AAFF15E0707847067F0E3800C0B235
S113B710002809D168467E210170477002226946DB
S113B7202000FFF782FF04E012223E212000FFF7F1
S113B73093FFF7BDF0B587B0254802902548264908
S113B7400691264901912649264A0592264A274B05
S113B7500493274B0093274B274C0394069C844265
S113B76007D00478029D2C70029C641C0294401C37
S113B770F4E7059C8C4207D00C78019D2C70019C49
S113B780641C0194491CF4E7049C944203D00024F3
S113B7901470521CF8E7039C9C4207D01C78009D4F
S113B7A02C705B1C009C641C0094F4E70024134D73
S113B7B0AD08AC4207D2124DA600AD59114EA700F8
S113B7C0F551641CF3E70F4D0F4E356007B0F0BD23
S113B7D0180800206CB30000C8B40000000000206A
S113B7E0B0860000C48E0000081600200D2E002034
S113B7F00000000000000000000000000000000045
S113B800000000000000000008ED00E0100201014B
S113B8100101010101000000D5AD00001102010188
S113B8200101010101000000C1B200002702010072
S113B8300000010001000000FD9600002803010043
S113B8400001010000000000B5A900003E02010152
S113B8500101010101000000D1B6000085020100D0
S113B86000010100000000007DB50000220300007B
S113B870010001000100000035A200002E040000B8
S113B8800000010001000000D5AB000031040100FC
S113B8900000010001000000C19100003405000017
S113B8A0000000000100000079A50000360200003D
S113B8B00000000001000000D3A7000037010000D1
S113B8C0000000000100000061B1000072B6002118
S113B8D0002200230024002500260027B846B9468C
S113B8E0BA46BB46BC460A490A4A521A013A05DD21
S113B8F00020042308601944043AFBDA064885460C
S113B900064880470648804762B6FAF731FCFEE7EE
S113B91000000020EF330020F0330020919D000050
S113B92035B70000000001003207000000010800E4
S113B93001000000FFFFFFFF01000100DF0700001E
S113B9400001080001000000FFFFFFFF02000100EA
S113B950B20700000000080000000000FFFFFFFF26
S113B9600300010034020000000008000000000091
S113B970FFFFFFFF0300011302401D010B0006003F
S113B980070008000C001C00180017040E000F40EC
S113B99004033D0121503E543F4C3C052300240048
S113B9A0250026002700280029002A002C002D004D
S113B9B02E002F0030003100320033002B00340001
S113B9C00000000070B40123002413E00168001D8E
S113B9D0194202D04D466918491E0C60091D121FF8
S113B9E0042AFAD20D00960701D50C80AD1C1A402A
S113B9F000D02C700268001D002AE7D170BC70478B
S113BA004669727374206672616D652073686F7520
S113BA106C64206E6F7420757365206D756C746929
S113BA20706C65206672616D65207472616E736DF1
S113BA30697373696F6E2E004D756C74692D66722F
S113BA40616D6520726573706F6E736520746F6FBE
S113BA50206C6172676520666F7220726563656928
S113BA6076696E67206275666665722E0000000056
S113BA704D6573736167652073697A6520746F6FB0
S113BA80206C617267652E205365742061206C619F
S113BA90726765722073656E64206275666665728E
S113BAA00A00000041626F72742070726576696FDB
S113BAB07573206D6573736167652C207472616E94
S113BAC0736D697373696F6E20696E2070726F672E
S113BAD0726573732E0A000059610000835F0000D1
S113BAE0CD5F000071600000D9600000ED600000CF
S113BAF001610000DF600000E7600000B301002086
S113BB00C1010020B5030020D1050020B784000046
S113BB109D84000081840000658400004984000045
S113BB202D840000558500003B8500001F85000022
S113BB3003850000E7840000CB84000053696E672E
S113BB406C652D6672616D65206C656E6774682026
S113BB50746F6F20736D616C6C206F7220746F6FE3
S113BB60206C617267652E00466972737420667278
S113BB70616D652073686F756C6420626520382080
S113BB80627974657320696E206C656E6774682EC3
S113BB900000000010B5074979441831064C7C4474
S113BBA0163404E0081D0A68891888470100A14278
S113BBB0F8D110BD2C000000380000000000000087
S113BBC00000000000000000000000000000000071
S113BBD00000000000000000000000000000000061
S113BBE0E5FDFFFF04000000001600200000000037
S113BBF0436F6E7365637574697665206672616DF3
S113BC006520746F6F2073686F72742E00000000DB
S113BC10466C6F7720636F6E74726F6C206672610E
S113BC206D6520746F6F2073686F72742E0000004E
S113BC3001000000020000000400000008000000F1
S113BC401000000020000000400000008000000000
S113BC5000F00DF8002801D0FFF79CFF00BF00BFE3
S113BC60002000BF00BFFAF783FA00F002F80120B9
S113BC70704780B500F002F801BD00000746384661
S113BC8000F002F8FBE7000080B500BF00BF024AE5
S113BC9011001820ABBEFBE7260002000548014650
S113BCA003B4684680F3098800BF00BF00BF00BF2B
S113BCB0FFF7CEFFA5EDF5FE30313233343536379C
S113BCC038394142434445466D61696E207374615D
S113BCD072740A00000102030405060708090A0B2E
S113BCE05465726D696E616C000000007101FF00A3
S113BCF0000000007101FF00000000007101020259
S113BD000000000053454747455200000102030468
S107BD104D535751E3
S903BC9DA3
